:100000000C94B2010C940F320C943C320C94DA0133
:100010000C94DA010C94DA010C94DA010C94DA01F4
:100020000C94DA010C94DA010C94DA010C94C506F4
:100030000C94DA010C94DA010C94DA010C94DA01D4
:100040000C941B310C94DA010C943B060C9477064B
:100050000C94DA010C94DA010C94DA010C94DA01B4
:100060000C94DA010C94DA01084AD73B3BCE016EBE
:1000700084BCBFFDC12F3D6C74319ABD56833DDAFF
:100080003D00C77F11BED9E4BB4C3E916BAAAABE0E
:10009000000000803F05A84CCDB2D44EB93836A937
:1000A000020C50B9918688083CA6AAAA2ABE000074
:1000B00000803F0664EC1B3C04BC163E3BE5B93CAB
:1000C000C93C37C29E5A3D660498083EEA69AAAA0E
:1000D0003E000000803F2020BF0020BF00BF007C0A
:1000E0002020202020202020202020202020202010
:1000F00020202000C8202020202020202020202078
:1001000020C900C8202020202020202020202020BE
:10011000C97C00D820202020202020202020202042
:10012000D97C00C820202020202020202020202032
:10013000C97C00C820202020202020202020202032
:10014000C97C00207265766F006D696E6F706F7389
:1001500064002020202020BABBBCBDBE7C20202013
:100160002020CACBCCCDCE7C00626F6F74696E67E5
:100170002075703AEDF2F2F2F2F2F2F2F3006261FF
:100180007474657279207761726E696E672000748D
:10019000787069642076616C756573006261726F56
:1001A0002074656D700074656D70646973702000F3
:1001B00061637469766520007061737369766500A8
:1001C00075617674616C6B20007365747570207353
:1001D000637265656E7C7C7C004368617220446F4D
:1001E0006E650A00526561647920666F7220466F01
:1001F0006E740A00557064617465204368617253BF
:1002000065740000407A10F35A00A0724E1809007D
:1002100010A5D4E80000E87648170000E40B54026B
:100220000000CA9A3B000000E1F5050000809698A6
:1002300000000040420F000000A0860100000010F6
:100240002700000000E80300000000640000000038
:10025000000A00000000000100000000002C76D819
:1002600088DC674F0823DFC1DFAE59E1B1B796E5FF
:10027000E3E453C63AE651997696E8E6C28426EB63
:10028000898C9B62ED407C6FFCEFBC9C9F40F2BA76
:10029000A56FA5F490055A2AF75C936B6CF9676D0E
:1002A000C11BFCE0E40D47FEF520E6B500D0ED9063
:1002B0002E0300943577050080841E080000204E30
:1002C0000A000000C80C333333330F986E128311C9
:1002D00041EF8D2114893BE65516CFFEE6DB18D1A0
:1002E000844B381BF77C1D901DA4BBE42420328472
:1002F000725E228100C9F124ECA1E53D276E616E9A
:1003000000696E660000000000240027002A00003B
:10031000000000250028002B00000000002300261C
:10032000002900040404040404040402020202027A
:1003300002030303030303010204081020408001A9
:100340000204081020010204081020000000070029
:10035000020100000304060000000000000000008D
:1003600046040C0811241FBECFEFD8E0DEBFCDBF7E
:1003700013E0A0E0B1E0E6ECFEE602C005900D92CD
:10038000AE3FB107D9F716E0AEEFB3E001C01D9262
:10039000A43BB107E1F713E0C4E6D3E004C0229721
:1003A000FE010E945D37C036D107C9F70E9426338F
:1003B0000C9461370C940000FA01AA27283051F1FF
:1003C000203181F1E8946F936E7F6E5F7F4F8F4F86
:1003D0009F4FAF4FB1E03ED0B4E03CD0670F781FE5
:1003E000891F9A1FA11D680F791F8A1F911DA11DCA
:1003F0006A0F711D811D911DA11D20D009F4689403
:100400003F912AE0269F11243019305D3193DEF6AA
:10041000CF010895462F4770405D4193B3E00FD060
:10042000C9F7F6CF462F4F70405D4A3318F0495D4B
:1004300031FD4052419302D0A9F7EACFB4E0A6952E
:100440009795879577956795BA95C9F70097610550
:10045000710508959B01AC010A2E069457954795A6
:1004600037952795BA95C9F7620F731F841F951F9B
:10047000A01D0895283008F027E03327DA01990FEE
:10048000311D87FD916000966105710539F4326078
:100490002E5F3D9330E32A95E1F708959F3F30F0BA
:1004A00080387105610509F03C5F3C5F3D939130F8
:1004B00008F08068911DDF93CF931F930F93FF92F5
:1004C000EF92192F987F9695E92F96959695E90FBB
:1004D000FF27E35AFD4F99273327EE24FF24A70176
:1004E000E70105900894079428F4360FE71EF81EDC
:1004F000491F511D660F771F881F991F0694A1F78A
:100500000590079428F4E70EF81E491F561FC11DD9
:10051000770F881F991F661F0694A1F7059007940F
:1005200028F4F80E491F561FC71FD11D880F991FA9
:10053000661F771F0694A1F70590079420F4490FD2
:10054000561FC71FD81F990F661F771F881F069455
:10055000A9F784911095177041F0D695C7955795D6
:100560004795F794E7941A95C1F7E3E0F2E06894B1
:100570001590159135916591959105907FE2739550
:10058000E118F10A430B560BC90BD009C0F7E10C77
:10059000F11E431F561FC91FD01D7EF4703311F486
:1005A0008A95E6CFE894015030F0080F0AF400274E
:1005B000021708F4202F2395022F7A3328F079E3CD
:1005C0007D932A95E9F710C07D932A9589F60694C4
:1005D00097956795379517951794E118F10A430B8E
:1005E000560BC90BD00998F023957E9173957A33F9
:1005F00008F070E37C932013B8F77E9170617D93CF
:1006000030F0839571E37D9370E32A95E1F711242F
:10061000EF90FF900F911F91CF91DF91992787FD68
:1006200090950895CF93DF93BC018230910510F42B
:1006300062E070E0A091B206B091B306ED0140E037
:1006400050E0E0E0F0E021C08881998186179707AB
:1006500069F48A819B81309719F09383828304C067
:100660009093B3068093B206FE0134C068177907F1
:1006700038F44115510519F08417950708F4AC01B9
:10068000FE018A819B819C01E9012097E9F64115D1
:100690005105A9F1CA01861B970B049708F4BA010A
:1006A000E0E0F0E02AC08D919C91119784179507A6
:1006B000F9F46417750781F412968D919C91139744
:1006C000309719F09383828304C09093B30680938C
:1006D000B206FD0132964CC0CA01861B970BFD0184
:1006E000E80FF91F6193719302978D939C9340C01B
:1006F000FD01828193819C01D9011097A1F680911F
:10070000B0069091B106892B41F480919F0290919F
:10071000A0029093B1068093B0064091A10250913F
:10072000A2024115510541F44DB75EB780919D027B
:1007300090919E02481B590B2091B0063091B10652
:10074000CA01821B930B8617970780F0AB014E5F9F
:100750005F4F8417950750F0420F531F5093B10617
:100760004093B006F9016193719302C0E0E0F0E0BC
:10077000CF01DF91CF910895CF93DF93009709F4D4
:1007800050C0EC0122971B821A82A091B206B09150
:10079000B306109709F140E050E0AC17BD0708F12F
:1007A000BB83AA83FE0121913191E20FF31FAE17A3
:1007B000BF0779F48D919C911197280F391F2E5FF7
:1007C0003F4F3983288312968D919C9113979B8379
:1007D0008A834115510571F4D093B306C093B206D4
:1007E00020C012968D919C911397AD01009711F046
:1007F000DC01D3CFFA01D383C28321913191E20F7F
:10080000F31FCE17DF0769F488819981280F391FFC
:100810002E5F3F4FFA01318320838A819B8193832E
:100820008283DF91CF910895FC0105906150704063
:100830000110D8F7809590958E0F9F1F0895FC01A9
:100840006150704001900110D8F7809590958E0FFF
:100850009F1F08956EBD0DB407FEFDCF8EB50895A0
:100860008DE061E00E9469328BE061E00E946932B4
:100870008CE060E00E9469328AE061E00E946932A7
:100880001CBC80E58CBD8DB58EB508958EEF93E0D0
:100890000E9430040895FC011382128288EE93E0D6
:1008A000A0E0B0E084839583A683B78383EB92E0D6
:1008B000918380830895FC018089803419F421E0BC
:1008C00030E002C020E030E0C9010895FC018189D8
:1008D00090E00895FC0164874587668747870895FF
:1008E00080E090E0089580E090E0089580E090E05E
:1008F00008950895EF92FF921F93CF93DF93162FE1
:100900007A0186E060E00E94A8328EEF93E060E01A
:100910000E942A048EEF93E060E00E942A048EEF8A
:1009200093E069E00E942A048EEF93E0612F0E9419
:100930002A04C0E0D0E0F701EC0FFD1F10818EEF1C
:1009400093E06AE00E942A048EEF93E06C2F0E94ED
:100950002A048EEF93E06BE00E942A048EEF93E06E
:10096000612F0E942A042196C633D10521F78EEF0C
:1009700093E068E00E942A048EEF93E060EA0E9410
:100980002A048EEF93E060EA0E942A0485FDF9CFE5
:100990008EEF93E060E00E942A048EEF93E06CE01B
:1009A0000E942A0486E061E00E94A832DF91CF9184
:1009B0001F91FF90EF9008951F93CF93DF93EC0169
:1009C000162F86E060E00E94A8328EEF93E060E090
:1009D0000E942A04112319F0113059F404C08EEF3B
:1009E00093E0688904C068896C618EEF93E00E948F
:1009F0002A0486E061E00E94A832DF91CF911F9126
:100A00000895EF92FF920F931F938EE1489F70011C
:100A10001124E60EF11C86E060E00E94A8320EEF81
:100A200013E0C80165E00E942A04C8016F2D0E94EE
:100A30002A04C80166E00E942A04C8016E2D0E94A3
:100A40002A041F910F91FF90EF900895EF92FF926B
:100A50000F931F937C010EEF13E0C80167E00E9423
:100A60002A04C8016FEF0E942A0486E061E00E9418
:100A7000A832F70187858F5F87871F910F91FF90BD
:100A8000EF900895EF92FF920F931F93FC01E7847C
:100A90008EE1E89E700111248685E80EF11C86E047
:100AA00060E00E94A8320EEF13E0C80164E00E94EB
:100AB0002A04C80163E00E942A04C80165E00E947C
:100AC0002A04C8016F2D0E942A04C80166E00E9412
:100AD0002A04C8016E2D0E942A041F910F91FF90D5
:100AE000EF9008951F93CF93DF93EC01162F6C378F
:100AF00031F40E942605CE010E9442050AC08EEF05
:100B000093E067E00E942A048EEF93E0612F0E9439
:100B10002A0481E090E0DF91CF911F9108950F9317
:100B20001F9386E060E00E94A8320EEF13E0C80138
:100B300064E00E942A04C80164E00E942A0486E05E
:100B400061E00E94A8321F910F9108951F93CF93E7
:100B5000DF93EC01188A16E0198B80EA96E060E9D1
:100B600073E00E947B30813049F480E4888B88E018
:100B7000898B86E060E00E94A83202C0188A198B37
:100B800086E060E00E94A832DF91CF911F91089526
:100B90000F931F93CF93DF93EC0186E061E00E94F7
:100BA000693282E060E00E94693282E061E00E9486
:100BB000A832CE010E94A60586E060E00E94A8321D
:100BC0008EEF93E06CEE0E942A048EEF93E06FEFBD
:100BD0000E942A04182F8EEF93E060E00E942A04FE
:100BE000688962608EEF93E00E942A0462E370E0FD
:100BF00080E090E00E9471318EEF93E06CE60E94FD
:100C00002A041F7E8EEF93E0612F0E942A048889B8
:100C1000803419F00DE010E002C000E110E0109205
:100C200000041092FF0317C06091FF03709100044D
:100C3000605F8EEF93E00E942A048EEF93E069E0FC
:100C40000E942A048091FF039091000401969093E2
:100C500000048093FF038091FF03909100048017AC
:100C6000910714F3CE0161E00E94DC04DF91CF9183
:100C70001F910F9108951F920F920FB60F9211249A
:100C80002F933F934F938F939F93EF93FF934091B5
:100C9000C60020918F06309190062F5F3F4F8091C4
:100CA0009306909194062823392380919106909180
:100CB00092062817390779F080918F069091900657
:100CC000E0919506F0919606E80FF91F4083309366
:100CD000900620938F06FF91EF919F918F914F91F6
:100CE0003F912F910F900FBE0F901F9018951F925C
:100CF0000F920FB60F9211242F933F938F939F93D0
:100D0000EF93FF932091990630919A068091970670
:100D10009091980628173907E9F0809199069091EB
:100D20009A06E0919D06F0919E06E80FF91F8081DA
:100D30008093C6008091990690919A060196209121
:100D40009B0630919C068223932390939A0680936E
:100D5000990610C0209197063091980680919906C7
:100D600090919A062817390729F48091C1008F7D48
:100D70008093C100FF91EF919F918F913F912F91AF
:100D80000F900FBE0F901F9018951F920F920FB6E5
:100D90000F9211248F939F938091C1049091C2046C
:100DA000892B51F08091C3049091C40401969093D3
:100DB000C4048093C30409C08091C5049091C60403
:100DC00001969093C6048093C5049F918F910F90D4
:100DD0000FBE0F901F901895CF93DF93482FEB0114
:100DE00080912606833009F45DC0843028F4813078
:100DF000C1F0823058F50AC0853009F4D2C0853080
:100E000008F4A8C0863009F0F2C0E9C04C3309F0FC
:100E1000EEC081E080932606488384EB809325060C
:100E2000E6C0842F90E0E0912506F0E0E827F9275E
:100E3000EF53FD4F208120932506887F9070809787
:100E400041F582E080932606498329C0242F30E0B3
:100E5000E0912506F0E0E227F327EF53FD4F808174
:100E600080932506809124068F5F8093240682302C
:100E700018F43B832A83BBC0922F88272A813B81A9
:100E8000820F931F9B838A830A978F3F910521F0DE
:100E900018F010922606ABC083E0809326061092CD
:100EA0002406A5C0E42FF0E08091250690E0E82715
:100EB000F927EF53FD4F808180932506609124062A
:100EC0006F5F60932406623089F0633020F46130F4
:100ED00009F08DC006C0633091F0643009F087C01E
:100EE00022C0842F90E0A0E0B0E018C0242F30E0B2
:100EF00040E050E0542F432F322F222707C0242FE9
:100F000030E040E050E0A901332722278C819D8109
:100F1000AE81BF81820F931FA41FB51F8C839D8359
:100F2000AE83BF8364C0242F30E040E050E0522FF6
:100F30004427332722278C819D81AE81BF81820F78
:100F4000931FA41FB51F8C839D83AE83BF836093C3
:100F50002606A5CF242F30E0E0912506F0E0E22719
:100F6000F327EF53FD4F808180932506809124065F
:100F70008F5F80932406813019F08230C1F503C061
:100F80003987288734C0922F882728853985280FEC
:100F9000391F398728878A819B810A97F1F085E07C
:100FA0007CCFE42FF0E08091250690E0E827F92738
:100FB000EF53FD4F808180932506209124062F5FFB
:100FC0002093240630E0FB01E20FF31F41878A8162
:100FD0009B810A972817390750F086E05ECFC75FDC
:100FE000DE4F4883C950D14087E080932606809128
:100FF0002606873069F410922606C75FDE4F90916F
:1010000025068881C950D140981711F48A8101C002
:1010100080E0DF91CF9108958F92AF92CF92EF92BF
:10102000FF920F931F9387E894E060E045EC50E057
:1010300024EC30E000EC10E0B1ECEB2EF12CCC24F1
:10104000C394A8E9AA2EF0E28F2E0E94EB2984EA2D
:1010500094E00E944B041092B7041092B8041092CE
:10106000B9041092BA041092BB041092BC041092FE
:10107000BD041092BE041092C0041092BF041092DE
:10108000B6041F910F91FF90EF90CF90AF908F908B
:101090000895AF92BF92CF92DF92EF92FF920F939B
:1010A0001F93E0908B06F0908C0600918D061091B6
:1010B0008E068FE590E0A0E0B0E0E80EF91E0A1F72
:1010C0001B1F0E9463316E157F058007910708F48E
:1010D0004EC0A090EC04B090ED04C090EE04D0900F
:1010E000EF04C601B50120E030E040E85FE30E9474
:1010F000C635181694F5E0904306F090440600912A
:101100004506109146060E94633120918B0630916E
:101110008C0640918D0650918E06621B730B840BDA
:10112000950B0E949C349B01AC01C601B5010E9445
:10113000D13520E030E04AE754E40E9403349B01BB
:10114000AC01C801B7010E94363360934306709327
:10115000440680934506909346060E94633160934F
:101160008B0670938C0680938D0690938E061F914C
:101170000F91FF90EF90DF90CF90BF90AF900895C8
:10118000DF93CF9300D000D0CDB7DEB7FB01E80FDF
:10119000F91F628583859485258569838A839B836E
:1011A0002C83492F5C81782FCA010F900F900F90EC
:1011B0000F90CF91DF910895AF92BF92DF92EF929F
:1011C000FF920F931F93CF93DF938C01809127069B
:1011D00080FDE4C0F801F08087E894E06F2D0E9464
:1011E000CC2AE801C75FDE4FEF2DF0E0EF53FD4F53
:1011F00080818883F801F18087E894E06F2D0E9458
:10120000CC2AEF2DF0E0888190E0E827F927EF5312
:10121000FD4F80818883F801F28087E894E06F2D8C
:101220000E94CC2AEF2DF0E0888190E0E827F92792
:10123000EF53FD4F80818883F801F38087E894E0C5
:101240006F2D0E94CC2AEF2DF0E0888190E0E827F6
:10125000F927EF53FD4F80818883F801F48087E8F8
:1012600094E06F2D0E94CC2AEF2DF0E0888190E071
:10127000E827F927EF53FD4F80818883F801248107
:10128000358146815781232F342F452F5527F22E44
:1012900087E894E0622F0E94CC2AEF2DF0E088814D
:1012A00090E0E827F927EF53FD4F80818883F8010C
:1012B00024813581468157819A0144275527F22E92
:1012C00087E894E0622F0E94CC2AEF2DF0E088811D
:1012D00090E0E827F927EF53FD4F80818883F801DC
:1012E0002481358146815781252F3327442755276F
:1012F000F22E87E894E0622F0E94CC2AEF2DF0E0D6
:10130000888190E0E827F927EF53FD4F808188839B
:1013100087E894E060E00E94CC2AE881F0E0EF5397
:10132000FD4F8081888387E894E060E00E94CC2AAA
:10133000E881F0E0EF53FD4F80818883F8018281DE
:1013400093810B9718F18AE0A82EB12CA00EB11E44
:10135000750112C0F701D1907F0187E894E06D2DEF
:101360000E94CC2AED2DF0E0888190E0E827F92753
:10137000EF53FD4F808188832E2D2A1930E0F8012C
:10138000828193810A972817390720F3075F1E4F40
:1013900087E894E0F80160810E94CC2ADF91CF9128
:1013A0001F910F91FF90EF90DF90BF90AF90089545
:1013B000DF93CF93CDB7DEB7CA50D1400FB6F894C4
:1013C000DEBF0FBECDBF2CE329836A832AE030E065
:1013D0003C832B83FC0184819581A681B7818D8319
:1013E0009E83AF83B887CE0101960E94DC08C65F5A
:1013F000DE4F0FB6F894DEBF0FBECDBFCF91DF91A9
:10140000089580EA96E06AE773E00E947B308823C3
:1014100031F586E696E6A6E6B0E48093280690933A
:101420002906A0932A06B0932B0680E090E0A0E85E
:10143000BFE380932C0690932D06A0932E06B093C5
:101440002F0688EE93E0909331068093300681E872
:10145000809332068DE8809333068DEF25C082E5B8
:1014600098EBAEE0B0E48093280690932906A09311
:101470002A06B0932B0685E89BEEA1E5B0E48093A5
:101480002C0690932D06A0932E06B0932F0680EA8B
:1014900094E190933106809330068BEF809332066F
:1014A00086E6809333068AEF809334060895FF9290
:1014B0000F931F9300EA16E0C8016CE773E00E94E7
:1014C0007B3080936F06C8016EE773E00E947B302B
:1014D00080937006C80160E873E00E947B308093BF
:1014E0004F06C8016EE873E00E947B308093670668
:1014F000C8016AE873E00E947B3080936506C801EA
:1015000064E873E00E947B3080937106C80166E84E
:1015100073E00E947B3080937206C8016CE873E030
:101520000E947B3080935706C80162E973E00E94F5
:101530007B3080937306C80164E973E00E947B30BE
:1015400080935606C80164EF73E00E947B30F82E4A
:10155000C80165EF73E00E947B30382F20E02F0D2B
:10156000311D3093750620937406C80166EF73E051
:101570000E947B30F82EC80167EF73E00E947B3039
:10158000382F20E02F0D311D3093770620937606FB
:10159000C80168EF73E00E947B30F82EC80169EF44
:1015A00073E00E947B30382F20E02F0D311D3093E7
:1015B000790620937806C8016BEF73E00E947B30B8
:1015C00080934E061F910F91FF900895BC0180EA11
:1015D00096E00E947B3008956091D6047091D70404
:1015E0008091D8049091D90420E030E040E152E4A9
:1015F0000E94D13520E030E044EB53E40E940334F4
:101600000E9434360E946B349B012550304037FFD6
:1016100003C09B01215E3F4FA7E3B6E0F901EF5302
:10162000FC4F80818C932F5F3F4F2432310514F0A3
:1016300020E030E0119686E0A234B80779F71C92DA
:1016400008952F923F924F925F926F927F928F9266
:101650009F92AF92BF92CF92DF92EF92FF920F9341
:101660001F93DF93CF9300D000D000D0CDB7DEB76B
:10167000182F662E2091CC043091CD042A353105E7
:1016800030F0C9018D549F4F89359105E8F437FF3B
:1016900002C02D543F4FC90137FF03C0909581957B
:1016A0009F4F8A3191053CF0F4E48F2E912CE9EDA7
:1016B0002E2E312C1DC00A975CF17BE3872E912CD6
:1016C00062ED262E312C20C02B35310514F0235B22
:1016D0003040C90137FF03C0909581959F4F8A31F3
:1016E000910554F056E5852E912C4CED242E312C8D
:1016F00037E0A32EB12C15C00A9754F02DE4822EAA
:10170000912C94ED292E312C88E0A82EB12C09C003
:1017100005E0802E912CB8E32B2E312CA9E0AA2EC7
:10172000B12C6091CE047091CF04882777FD80950D
:10173000982F0E949E3427EA32E94BE25CEB0E942C
:10174000D1350E94A53620E030E040EA50E40E9406
:10175000D13520E030E040E951E40E94D1350E94CB
:10176000343620E030E044E352E40E9436330E94F5
:101770006B34712EFEEBCF2EFFEFDF2E9B01442743
:1017800037FD4095542F29833A834B835C83E4EAE9
:101790004E2EE4E05E2E4AEF5FEF240E351E609180
:1017A000CC047091CD04882777FD8095982F0E94F6
:1017B0009E3425E33AEF4EE85CE30E94D1350E9467
:1017C000A5367B018C01B601882777FD8095982F7F
:1017D0000E949E349B01AC01C801B7010E94D13523
:1017E0007B018C0169817A818B819C810E949E346E
:1017F0009B01AC01C801B7010E9436330E946B34D3
:101800009B01CB0101978A35910508F071C062E117
:1018100070E00E940B378B012F5F3F4FAEEEBFEFA2
:101820006A9FC0016B9F900D7A9F900D1124820FCB
:10183000931F62E070E00E940B376D837E83E62C7D
:10184000E01A4E2D4C5F84EA94E0672D0E9401055A
:1018500000D000D000D0EDB7FEB73196ADB7BEB71F
:1018600012965C924E92119720E031E033832283EE
:101870008D819E81880D991D958384830E94CA293C
:101880004DB75EB74A5F5F4F0FB6F8945EBF0FBEAD
:101890004DBF8D819E818A159B0554F10430110541
:1018A0003CF593E0E90EC201672D4E2D0E94010523
:1018B00000D000D000D0EDB7FEB73196ADB7BEB7BF
:1018C00012965C924E92119720E031E0338322838E
:1018D0004D815E81420D531D558344830E94CA2968
:1018E0008DB79EB706960FB6F8949EBF0FBE8DBFFC
:1018F000ACE0B0E0CA0EDB1E7394BEE4CB16D1049C
:1019000009F04DCF26960FB6F894DEBF0FBECDBFBF
:10191000CF91DF911F910F91FF90EF90DF90CF90CB
:10192000BF90AF909F908F907F906F905F904F90FF
:101930003F902F900895823010F422E002C0282FAB
:10194000220F30E08DB79EB708970FB6F8949EBF70
:101950000FBE8DBFEDB7FEB7319684EA94E0ADB708
:10196000BEB712969C938E93119783E091E0938378
:10197000828322573F4F358324832F5F3F4F378326
:1019800026830E94CA298DB79EB708960FB6F89491
:101990009EBF0FBE8DBF0895CF93DF93AC01E09142
:1019A000DE04F091DF042091350630913606C9013E
:1019B0008C599F4F8E179F071CF4EA01219709C08D
:1019C00024563040E217F30714F0EA0102C0EA019E
:1019D0002196842F90E0C817D90729F080EA96E075
:1019E0004C2F0E948230CE01DF91CF9108950F934A
:1019F0001F9300EA16E0C80163EF73E041E00E9424
:101A00008230C80164EF73E043E10E948230C80174
:101A100065EF73E046E00E948230C80166EF73E034
:101A200040E10E948230C80167EF73E047E20E9404
:101A30008230C80168EF73E048E80E948230C80134
:101A400069EF73E043E10E9482301F910F91089586
:101A5000CF92DF92EF92FF920F931F937C01D62ECD
:101A6000C72E04EA14E0C8016E2D4D2D0E946A04B1
:101A7000C8010E94420500D000D0EDB7FEB7128326
:101A8000018383E391E0948383830E94B929EDB7B6
:101A9000FEB71283018383E291E0948383830E94E3
:101AA000B929EDB7FEB71283018383E191E09483F6
:101AB00083830E94B929EDB7FEB71283018383E0C7
:101AC00091E0948383830E94B929EDB7FEB7128316
:101AD000018384EF90E0948383830E94B9290F905F
:101AE0000F900F900F90C8010E942605C701019624
:101AF0006D2D7C2D0E94210B1F910F91FF90EF9077
:101B0000DF90CF900895CF92DF92EF92FF920F93E4
:101B10001F93CF93DF93182F062F0E94633128EE77
:101B200033E040E050E00E941E3769017A01C4EAC8
:101B3000D4E0CE01612F402F0E946A04CE010E94A2
:101B400042058091FE049091FF04892B09F453C053
:101B500000910005109101058DB79EB744970FB60F
:101B6000F8949EBF0FBE8DBFEDB7FEB73196ADB7EF
:101B7000BEB71296DC93CE93119788E091E09383E1
:101B8000828383EB90E095838483C6016CE370E0ED
:101B90000E940B37CB016CE370E00E940B379783F8
:101BA00086832AE330E031872087C6016CE370E04A
:101BB0000E940B379387828785E690E0958784871C
:101BC000C8016CE370E00E94F736CB016CE370E073
:101BD0000E940B3797878687318B208BC8016CE377
:101BE00070E00E94F736938B828B0E94CA298DB7D2
:101BF0009EB7449633C0ADB7BEB71C970FB6F894E6
:101C0000BEBF0FBEADBFEDB7FEB731961296DC93E7
:101C1000CE93119780E291E09383828383EB90E0EF
:101C200095838483C6016CE370E00E940B37CB017F
:101C30006CE370E00E940B37978386838AE390E021
:101C400091878087C6016CE370E00E940B37938711
:101C500082870E94CA298DB79EB70C960FB6F8945A
:101C60009EBF0FBE8DBF84EA94E00E942605DF91DF
:101C7000CF911F910F91FF90EF90DF90CF9008953B
:101C8000EF92FF920F931F93282F462FA4EAEA2E7C
:101C9000A4E0FA2EC701622F0E946A04C7010E94C5
:101CA00042058DB79EB70A970FB6F8949EBF0FBE38
:101CB0008DBF0DB71EB70F5F1F4FEDB7FEB7F28296
:101CC000E1828CE291E0F8019383828360910205C6
:101CD00070910305809104059091050520912C06D3
:101CE00030912D0640912E0650912F060E94D1353D
:101CF000F801648375838683978380EB90E09187F6
:101D000080870E94CA298DB79EB70A960FB6F894AD
:101D10009EBF0FBE8DBFC7010E9426051F910F9168
:101D2000FF90EF9008958F929F92AF92BF92CF92C3
:101D3000DF92EF92FF920F931F93E82EF62E04EAA4
:101D400014E0C8016E2D4F2D0E946A04C8010E9444
:101D500042058DB79EB70C970FB6F8949EBF0FBE85
:101D60008DBFEDB7FEB73196ADB7BEB712961C93D7
:101D70000E93119794E3892E91E0992E938282829B
:101D80008DEEA82EB12CB582A48280910B05909186
:101D90000C05A0910D05B0910E0586839783A08751
:101DA000B187B3EFCB2ED12CD386C2860E94CA292D
:101DB0008DB79EB70C960FB6F8949EBF0FBE8DBF21
:101DC000C8010E942605F394C8016E2D4F2D0E9474
:101DD0006A04C8010E944205ADB7BEB71C970FB692
:101DE000F894BEBF0FBEADBFEDB7FEB731961296E9
:101DF0001C930E93119793828282B582A482809164
:101E00000F0590911005A0911105B09112058683E0
:101E10009783A087B187D386C2860E94CA298DB7CF
:101E20009EB70C960FB6F8949EBF0FBE8DBFC8012B
:101E30000E942605F394C8016E2D4F2D0E946A045E
:101E4000C8010E944205ADB7BEB71C970FB6F89403
:101E5000BEBF0FBEADBFEDB7FEB7319612961C9355
:101E60000E93119793828282B582A482809113058A
:101E700090911405A0911505B0911605868397835E
:101E8000A087B187D386C2860E94CA298DB79EB724
:101E90000C960FB6F8949EBF0FBE8DBFC8010E946E
:101EA00026051F910F91FF90EF90DF90CF90BF908C
:101EB000AF909F908F9008950F931F93282F462FD8
:101EC00004EA14E0C801622F0E946A04C8010E945B
:101ED00042058DB79EB70A970FB6F8949EBF0FBE06
:101EE0008DBFEDB7FEB73196ADB7BEB712961C9356
:101EF0000E9311978EE391E09383828389EB90E0B8
:101F0000958384838091FE049091FF049783868358
:101F100082E890E0918780870E94CA298DB79EB79A
:101F20000A960FB6F8949EBF0FBE8DBFC8010E94DF
:101F300026051F910F910895EF92FF920F931F9323
:101F4000282F462F34EAE32E34E0F32EC701622F08
:101F50000E946A04C7010E9442058DB79EB70C9784
:101F60000FB6F8949EBF0FBE8DBF0DB71EB70F5FA3
:101F70001F4FEDB7FEB7F282E18286E491E0F801EF
:101F80009383828384EE90E0958384836091FC0444
:101F90007091FD04882777FD8095982F0E949E34CC
:101FA0002AE037ED43E25CE30E94D135F801668315
:101FB0007783808791878FE890E0938782870E945C
:101FC000CA298DB79EB70C960FB6F8949EBF0FBE68
:101FD0008DBFC7010E9426051F910F91FF90EF90C2
:101FE00008950F931F93282F462F04EA14E0C80189
:101FF000622F0E946A04C8010E9442058DB79EB7F5
:102000000C970FB6F8949EBF0FBE8DBFEDB7FEB70D
:102010003196ADB7BEB712961C930E93119786E416
:1020200091E09383828382EE90E095838483809114
:10203000F8049091F904A091FA04B091FB0486830E
:102040009783A087B1878EE890E0938782870E946C
:10205000CA298DB79EB70C960FB6F8949EBF0FBED7
:102060008DBFC8010E9426051F910F9108950F93FF
:102070001F93282F462F84EA94E0622F0E946A045F
:1020800084EA94E00E9442058091DB04882319F4DD
:1020900020E531E057C0813019F424E531E052C029
:1020A000823019F428E531E04DC0833019F42CE575
:1020B00031E048C0843019F420E631E043C0853077
:1020C00019F424E631E03EC0863019F428E631E008
:1020D00039C0873019F42CE631E034C0883019F467
:1020E00020E731E02FC0893019F424E731E02AC01D
:1020F0008A3019F428E731E025C08B3019F42CE739
:1021000031E020C08C3019F420E831E01BC08D3064
:1021100019F424E831E016C08E3019F428E831E0D3
:1021200011C08F3019F42CE831E00CC0803119F463
:1021300020E931E007C0813119F024E931E002C023
:1021400025E931E08DB79EB708970FB6F8949EBF8A
:102150000FBE8DBFEDB7FEB7319604EA14E0ADB700
:10216000BEB712961C930E93119789E991E0938361
:10217000828380EE90E095838483378326830E9458
:10218000CA298DB79EB708960FB6F8949EBF0FBEAA
:102190008DBFC8010E9426051F910F9108950F93CE
:1021A0001F93282F462F04EA14E0C801622F0E94D3
:1021B0006A04C8010E9442058DB79EB70A970FB600
:1021C000F8949EBF0FBE8DBFEDB7FEB73196ADB789
:1021D000BEB712961C930E9311978EE991E09383EC
:1021E000828387E890E0958384838091DC049091DA
:1021F000DD049783868385E290E0918780870E9443
:10220000CA298DB79EB70A960FB6F8949EBF0FBE27
:102210008DBFC8010E9426051F910F9108950F934D
:102220001F93282F462F04EA14E0C801622F0E9452
:102230006A04C8010E9442058DB79EB70A970FB67F
:10224000F8949EBF0FBE8DBFEDB7FEB73196ADB708
:10225000BEB712961C930E93119788EA91E0938370
:1022600082838091CE049091CF049583848380EB08
:1022700090E09783868381EB90E0918780870E942E
:10228000CA298DB79EB70A960FB6F8949EBF0FBEA7
:102290008DBFC8010E9426051F910F9108950F93CD
:1022A0001F93282F462F04EA14E0C801622F0E94D2
:1022B0006A04C8010E9442058DB79EB70A970FB6FF
:1022C000F8949EBF0FBE8DBFEDB7FEB73196ADB788
:1022D000BEB712961C930E93119788EA91E09383F0
:1022E00082838091CC049091CD049583848380EB8C
:1022F00090E09783868382EB90E0918780870E94AD
:10230000CA298DB79EB70A960FB6F8949EBF0FBE26
:102310008DBFC8010E9426051F910F9108950F934C
:102320001F93282F462F04EA14E0C801622F0E9451
:102330006A04C8010E9442058DB79EB70A970FB67E
:10234000F8949EBF0FBE8DBFEDB7FEB73196ADB707
:10235000BEB712961C930E93119780EB91E0938376
:10236000828381EE90E0958384838091AB0290918B
:10237000AC029783868385E290E0918780870E94F4
:10238000CA298DB79EB70A960FB6F8949EBF0FBEA6
:102390008DBFC8010E9426051F910F9108950F93CC
:1023A0001F93282F462F04EA14E0C801622F0E94D1
:1023B0006A04C8010E9442058DB79EB70C970FB6FC
:1023C000F8949EBF0FBE8DBFEDB7FEB73196ADB787
:1023D000BEB712961C930E93119788EB91E09383EE
:1023E000828382EC91E09583848380ED90E09783F3
:1023F000868387E396E09187808781ED90E09387DD
:1024000082870E94CA298DB79EB70C960FB6F894A2
:102410009EBF0FBE8DBFC8010E9426051F910F9160
:1024200008950F931F93282F462F04EA14E0C80144
:10243000622F0E946A04C8010E9442058DB79EB7B0
:102440000A970FB6F8949EBF0FBE8DBFEDB7FEB7CB
:102450003196ADB7BEB712961C930E93119780EDCF
:1024600091E0938382838091D6049091D704A091C8
:10247000D804B091D90484839583A683B78380EB75
:1024800090E0918780870E94CA298DB79EB70A96EF
:102490000FB6F8949EBF0FBE8DBFC8010E942605DF
:1024A0001F910F9108950F931F93282F462F04EA31
:1024B00014E0C801622F0E946A04C8010E9442050C
:1024C0008DB79EB70C970FB6F8949EBF0FBE8DBF09
:1024D000EDB7FEB73196ADB7BEB712961C930E930B
:1024E000119788ED91E09383828386E190E0958354
:1024F00084838091F0049091F104A091F204B09152
:10250000F30486839783A087B18788E890E0938758
:1025100082870E94CA298DB79EB70C960FB6F89491
:102520009EBF0FBE8DBFC8010E9426051F910F914F
:102530000895CF92DF92EF92FF920F931F93CF9364
:10254000DF93282F462FC4EAD4E0CE01622F0E94E9
:102550006A04CE010E9442056091430670914406D0
:10256000809145069091460620912C0630912D06CB
:1025700040912E0650912F060E94D1356B017C01AF
:1025800020E030E04AE754E40E94C6351816D4F53E
:102590008DB79EB70C970FB6F8949EBF0FBE8DBF38
:1025A0000DB71EB70F5F1F4FADB7BEB71296DC93C6
:1025B000CE93119786E491E0F801938382838EEFA6
:1025C00090E095838483609130067091310688276E
:1025D00077FD8095982F0E949E349B01AC01C70126
:1025E000B6010E940334D80116966D937D938D93A6
:1025F0009C931997809134061A968C931A971B9680
:102600001C9221C08DB79EB70C970FB6F8949EBF51
:102610000FBE8DBFEDB7FEB73196ADB7BEB7129600
:10262000DC93CE93119782EE91E0938382838EEFB9
:1026300090E095838483C682D782E086F18680917C
:102640003306828713860E94CA29EDB7FEB73C96EF
:102650000FB6F894FEBF0FBEEDBF84EA94E00E946F
:102660002605DF91CF911F910F91FF90EF90DF90A2
:10267000CF900895EF92FF920F931F93282F462F2C
:1026800054EAE52E54E0F52EC701622F0E946A0439
:10269000C7010E9442058DB79EB70C970FB6F894FC
:1026A0009EBF0FBE8DBF0DB71EB70F5F1F4FEDB79B
:1026B000FEB7F282E18288ED91E0F8019383828394
:1026C00089EE90E0958384836091EC047091ED0431
:1026D0008091EE049091EF04209128063091290614
:1026E00040912A0650912B060E94D135F80166834D
:1026F00077838087918780913206828713860E9434
:10270000CA298DB79EB70C960FB6F8949EBF0FBE20
:102710008DBFC7010E9426051F910F91FF90EF907A
:102720000895EF92FF920F931F93282F462F64EA8C
:10273000E62E64E0F62EC701622F0E946A04C701EC
:102740000E9442058DB79EB70C970FB6F8949EBFB6
:102750000FBE8DBF0DB71EB70F5F1F4FEDB7FEB792
:10276000F282E18288ED91E0F8019383828388EE22
:1027700090E0958384836091F4047091F5048091D6
:10278000F6049091F7042091280630912906409193
:102790002A0650912B060E94D135F8016683778373
:1027A0008087918780913206828713860E94CA298A
:1027B0008DB79EB70C960FB6F8949EBF0FBE8DBF17
:1027C000C7010E9426051F910F91FF90EF90089579
:1027D000EF92FF920F931F93282F462F74EAE72E54
:1027E00074E0F72EC701622F0E946A04C7010E949D
:1027F00042058DB79EB70C970FB6F8949EBF0FBEDB
:102800008DBF0DB71EB70F5F1F4FEDB7FEB7F2823A
:10281000E18282EE91E0F8019383828386EE90E07C
:10282000958384836091E8047091E9048091EA04BF
:102830009091EB0420912C0630912D0640912E06AC
:1028400050912F060E94D135F801668377838087E7
:10285000918780913306828713860E94CA298DB79B
:102860009EB70C960FB6F8949EBF0FBE8DBFC701E2
:102870000E9426051F910F91FF90EF900895EF920F
:10288000FF920F931F93282F462FE4EAEE2EE4E0E9
:10289000FE2EC701622F0E946A04C7010E944205F2
:1028A0008DB79EB70C970FB6F8949EBF0FBE8DBF25
:1028B0000DB71EB70F5F1F4FEDB7FEB7F282E18273
:1028C00082EE91E0F8019383828387EE90E0958316
:1028D00084836091060570910705882777FD8095B0
:1028E000982F0E949E3420912C0630912D06409105
:1028F0002E0650912F060E94D135F801668377830A
:102900008087918780913306828713860E94CA2927
:102910008DB79EB70C960FB6F8949EBF0FBE8DBFB5
:10292000C7010E9426051F910F91FF90EF90089517
:102930000F931F93282F462F04EA14E0C801622F3B
:102940000E946A04C8010E944205809147060E94C5
:102950009B0CC8010E9426051F910F910895EF92CC
:10296000FF920F931F93282F462FF4EAEF2EF4E0E7
:10297000FF2EC701622F0E946A04C7010E94420510
:102980008DB79EB70C970FB6F8949EBF0FBE8DBF44
:102990000DB71EB70F5F1F4FEDB7FEB7F282E18292
:1029A00082EE91E0F801938382838FE190E095833A
:1029B0008483609148067091490680914A069091FF
:1029C0004B060E949E3420912C0630912D0640919A
:1029D0002E0650912F060E94D135F8016683778329
:1029E0008087918780913306828713860E94CA2947
:1029F0008DB79EB70C960FB6F8949EBF0FBE8DBFD5
:102A0000C7010E9426051F910F91FF90EF90089536
:102A10000F931F93282F462F04EA14E0C801622F5A
:102A20000E946A04C8010E9442058DB79EB7409774
:102A30000FB6F8949EBF0FBE8DBFEDB7FEB73196AF
:102A4000ADB7BEB712961C930E9311978CEE91E022
:102A50009383828383E890E0958384838091D2047A
:102A60009091D304A091D404B091D5048683978328
:102A7000A087B18784E890E0938782878091E20401
:102A80009091E304A091E404B091E50484879587D4
:102A9000A687B7870E94CA298DB79EB740960FB602
:102AA000F8949EBF0FBE8DBFC8010E9426051F91DE
:102AB0000F9108950F931F93282F462F84EA94E0D7
:102AC000622F0E946A0484EA94E00E944205809189
:102AD000E704282F30E0823030F4A4E0220F331FC7
:102AE000AA95E1F702C02150304000D000D000D0BC
:102AF000EDB7FEB7319604EA14E0ADB7BEB7129653
:102B00001C930E93119780E091E093838283358329
:102B100024830E94CA298DB79EB706960FB6F894F3
:102B20009EBF0FBE8DBFC8010E9426051F910F9149
:102B300008950F931F93282F462F04EA14E0C8012D
:102B4000622F0E946A04C8010E9442058DB79EB799
:102B500008970FB6F8949EBF0FBE8DBFEDB7FEB7B6
:102B60003196ADB7BEB712961C930E9311978EEFA8
:102B700091E0938382838FE090E0958384838091BA
:102B8000E604868317820E94CA298DB79EB70896ED
:102B90000FB6F8949EBF0FBE8DBFC8010E942605D8
:102BA0001F910F9108950F931F9304EA14E0C80139
:102BB00063E045E00E946A04C8010E94420500D01B
:102BC00000D0EDB7FEB71283018382E591E09483D4
:102BD00083830E94B929EDB7FEB71283018389E48C
:102BE00091E0948383830E94B929EDB7FEB71283E5
:102BF000018383E491E0948383830E94B9290F9039
:102C00000F900F900F90C8010E9426051F910F9101
:102C100008950F931F93282F462F04EA14E0C8014C
:102C2000622F0E946A04C8010E94420500D000D0B1
:102C3000EDB7FEB71283018389E691E09483838325
:102C40000E94B9290F900F900F900F90C8010E9419
:102C500026051F910F910895EF92FF920F931F93F6
:102C6000CF93DF930E946331209151063091520639
:102C700040915306509154062617370748075907C5
:102C800008F08AC10E9463316C507E4F8F4F9F4F76
:102C900060935106709352068093530690935406A6
:102CA00004EA14E0C8010E948F05C80165E043E012
:102CB0000E946A04C8010E94420500D000D0EDB70E
:102CC000FEB71283018389EC91E0948383830E9491
:102CD000B9290F900F900F900F9080913506909129
:102CE0003606892B31F080914C0690914D06892B48
:102CF00081F48091DE049091DF04909336068093F6
:102D000035068091E0049091E10490934D06809304
:102D10004C062091E0043091E10440914C06509122
:102D20004D06C901845690404817590724F48091F4
:102D300050068F5F08C02C593F4F241735072CF4DD
:102D4000809150068150809350068091500618164D
:102D500014F081E003C084301CF083E080935006BF
:102D600080915006823009F462C0833009F4BEC0FD
:102D7000813009F00DC100D000D0C4EAD4E0EDB735
:102D8000FEB7D283C18380EC91E0948383830E9459
:102D9000B929809127060F900F900F900F9080FF18
:102DA00022C000D000D0EDB7FEB7D283C18388EB3C
:102DB00091E0948383830E94B92980913506909194
:102DC0003606845690400F900F900F900F902091F0
:102DD000DE043091DF04281739070CF0D9C0809148
:102DE00027068E7F21C000D000D0EDB7FEB7D2837A
:102DF000C18380EB91E0948383830E94B929809101
:102E00003506909136068C599F4F0F900F900F907A
:102E10000F902091DE043091DF04821793070CF0AD
:102E2000B7C080912706816080932706B1C000D08B
:102E300000D0C4EAD4E0EDB7FEB7D283C18386EAFE
:102E400091E0948383830E94B9290F900F900F9093
:102E50000F9080914E06882301F100D000D0EDB78D
:102E6000FEB7D283C1838CE991E0948383830E946F
:102E7000B9298091350690913606845690400F907E
:102E80000F900F900F902091DE043091DF042817EF
:102E900039071CF510924E0620C000D000D0EDB7C7
:102EA000FEB7D283C1838FE891E0948383830E942D
:102EB000B92980913506909136068C599F4F0F9015
:102EC0000F900F900F902091DE043091DF04821755
:102ED00093071CF481E080934E0680EA96E06BEF46
:102EE00073E040914E060E94823052C000D000D064
:102EF000B4EAEB2EB4E0FB2EEDB7FEB7F282E1822E
:102F00008EE791E0948383830E94B9298DB79EB7A1
:102F100008970FB6F8949EBF0FBE8DBF0DB71EB7B2
:102F20000F5F1F4FEDB7FEB7F282E18284E092E0BF
:102F3000F8019383828360914F0670E080E090E017
:102F40000E949C3420E030E040E251E40E940334CF
:102F5000F801648375838683978386E790E0918781
:102F6000808780E290E0938782870E94CA298DB78C
:102F70009EB70C960FB6F8949EBF0FBE8DBF809182
:102F80004F0690E060E873E00E94CC0C80934F06FF
:102F900084EA94E00E942605DF91CF911F910F9162
:102FA000FF90EF900895BF92CF92DF92EF92FF9241
:102FB0000F931F93CF93DF93E82ED62E0E94633199
:102FC00020915E0630915F06409160065091610647
:102FD000261737074807590708F024C18091620671
:102FE0008823C9F08093AD02109262068CE092E0D3
:102FF00090936406809363060E9463316C507E4F09
:103000008F4F9F4F60935E0670935F0680936006BC
:1030100090936106C2C08091AD02A82FB0E070917C
:10302000DA044091630650916406F090C704109151
:10303000E7040091550660911805E091AB02F0910C
:10304000AC0280915606C82FD0E0B0905706909100
:1030500017059D012F5F3F4F273031051CF021E000
:1030600030E019C02330310531F12430310544F40A
:103070002130310581F02230310509F057C012C0EE
:103080002530310591F125303105ECF02630310540
:1030900009F04CC037C0723008F048C049E152E036
:1030A00081E049C083E0C82EFC1409F43FC046E229
:1030B00052E082E040C01230C8F50023B9F143E38A
:1030C00052E083E038C0623088F1633039F0643018
:1030D00041F0623041F440E452E005C04DE452E07A
:1030E00002C04AE552E084E026C0EC17FD07F4F484
:1030F0008FEFED39F807D1F0BB20C1F447E652E07D
:1031000085E019C0723090F4923080F0933039F03D
:10311000943041F0923051F444E752E005C040E869
:1031200052E002C04DE852E086E005C02A173B0796
:1031300009F090CF60C0509364064093630680937B
:10314000620681E0809358060E94633168517C4F8B
:103150008F4F9F4F60935E0670935F06809360066B
:10316000909361060E9463316056704F8F4F9F4F5E
:1031700060935A0670935B0680935C0690935D069D
:1031800080915906882321F084EA94E00E948F05FB
:103190001092590602C01092580604EA14E0C801C1
:1031A0006E2D4D2D0E946A04C8010E94420500D078
:1031B00000D000D0EDB7FEB73196ADB7BEB71296CE
:1031C0001C930E9311978AE992E0938382838091F6
:1031D000630690916406958384830E94CA298DB703
:1031E0009EB706960FB6F8949EBF0FBE8DBFC8015E
:1031F0000E94260517C05093640640936306109200
:1032000062060E94633120915A0630915B0640911C
:103210005C0650915D06261737074807590708F4E2
:10322000BACFBBCFDF91CF911F910F91FF90EF905D
:10323000DF90CF90BF900895EF92FF920F931F936E
:1032400080916506843009F056C09091DB0494307B
:1032500008F027C180916E068917A1F190936E0640
:103260000E94633160936A0670936B0680936C06CC
:1032700090936D0690916E068091AE02981711F5AD
:1032800080915906813091F0813018F08230B1F48C
:1032900013C011E0109359060E94633161537547C2
:1032A0008040904030F41093660608C082E080931E
:1032B00059061092660602C01092590684EA94E0FC
:1032C0000E948F050E94633120916A0630916B063F
:1032D00040916C0650916D06621B730B840B950B2D
:1032E000615D77408040904008F4DBC08091DB0452
:1032F0008093AE02D6C0853029F48091A3029091CC
:10330000A40214C0863029F48091A5029091A602EF
:103310000DC0873029F48091A7029091A80206C0C1
:10332000883041F48091A9029091AA029093690695
:10333000809368068091670620916806309169063F
:10334000882309F04AC0C901895097408F5A944098
:10335000C8F40E946331615375478040904020F467
:1033600081E0809366060CC080916606882341F454
:1033700080915806882321F484EA94E00E948F0506
:1033800082E028C044E0203B340768F4809159066D
:10339000882349F01092660684EA94E00E948F0523
:1033A000109259067EC0205B34402955324008F007
:1033B00078C080915906813009F473C08091580615
:1033C000882309F06EC01092660684EA94E00E9499
:1033D0008F0581E08093590664C0215B344008F476
:1033E00060C00E946331615375478040904008F08F
:1033F00041C0809166068823E9F5E0906A06F09066
:103400006B0600916C0610916D0688EE93E0A0E0CB
:10341000B0E0E80EF91E0A1F1B1F0E946331E6167A
:10342000F70608071907E8F581E08093660617C0DC
:103430001092660684EA94E00E948F0580915906F6
:10344000823019F41092590603C08F5F8093590699
:1034500080915906823018F082E0809359060E94CC
:10346000633160936A0670936B0680936C06909349
:103470006D0617C0E0906A06F0906B0600916C062E
:1034800010916D0688EE93E0A0E0B0E0E80EF91E22
:103490000A1F1B1F0E946331E616F706080719076B
:1034A00038F21F910F91FF90EF900895809165067B
:1034B000843010F00E941C1980916606882319F050
:1034C0000E942C1608958091070480FF08C0609127
:1034D0006D0480916B0490E070E00E94D31780919E
:1034E0005906823008F012C2A82FB0E0FD01EF5F4C
:1034F000FB4F808185FF0BC0FD01E35EFB4F6081C8
:10350000A55EBB4F8C9190E070E00E949915809170
:103510005906A82FB0E0FD01EF5FFB4F808186FFC9
:103520000BC0FD01EF5DFB4F6081A15EBB4F8C9135
:1035300090E070E00E945A1580915506882309F4A6
:103540003FC080915906A82FB0E0FD01EF5FFB4F0F
:10355000808187FF0BC0FD01EB5DFB4F6081AD5D9E
:10356000BB4F8C9190E070E00E9408158091590645
:10357000A82FB0E0FD01ED5FFB4F808184FF0BC001
:10358000FD01E35CFB4F6081A55CBB4F8C9190E03B
:1035900070E00E94AF1480915906A82FB0E0FD01A1
:1035A000ED5FFB4F808183FF0BC0FD01E75CFB4FAC
:1035B0006081A95CBB4F8C9190E070E00E949814F0
:1035C00080915906A82FB0E0FD01EB5FFB4F808191
:1035D00087FF0BC0FD01EB5AFB4F6081AD5ABB4F1B
:1035E0008C9190E070E00E943F1480915906A82FC2
:1035F000B0E0FD01E95FFB4F808183FF0BC0FD015F
:10360000EB58FB4F6081AD58BB4F8C9190E070E060
:103610000E94531280915906A82FB0E0FD01EB5F84
:10362000FB4F808181FF0BC0FD01E35AFB4F60819E
:10363000A55ABB4F8C9190E070E00E94911380914D
:103640005506882309F444C08091E704823008F4C9
:103650003FC080915906A82FB0E0FD01E75FFB4F06
:10366000808182FF0BC0FD01EF57FB4F6081A158A5
:10367000BB4F8C9190E070E00E94991280915906A6
:10368000A82FB0E0FD01EB5FFB4F808182FF0BC0F4
:10369000FD01EF5AFB4F6081A15BBB4F8C9190E025
:1036A00070E00E94E81380915906A82FB0E0FD0158
:1036B000EB5FFB4F808183FF0BC0FD01E75AFB4F9F
:1036C0006081A95ABB4F8C9190E070E00E943A1340
:1036D00080915906A82FB0E0FD01ED5FFB4F80817E
:1036E00081FF0BC0FD01EF5CFB4F6081A15DBB4F13
:1036F0008C9190E070E00E94111280915906A82FE1
:10370000B0E0FD01ED5FFB4F808180FF0BC0FD014C
:10371000E35DFB4F6081A55DBB4F8C9190E070E055
:103720000E94CF1180915906A82FB0E0FD01E95FFA
:10373000FB4F808186FF0BC0FD01E358FB4F60818A
:10374000A558BB4F8C9190E070E00E948F11809142
:103750005906A82FB0E0FD01EF5FFB4F808182FF8B
:103760000BC0FD01EB5EFB4F6081AD5EBB4F8C91EA
:1037700090E070E00E944F1180915906A82FB0E0B0
:10378000FD01EF5FFB4F808181FF0BC0FD01EF5E0C
:10379000FB4F6081A15FBB4F8C9190E070E00E9475
:1037A0000F1180915906A82FB0E0FD01EB5FFB4F90
:1037B000808184FF0BC0FD01EF59FB4F6081A15A4E
:1037C000BB4F8C9190E070E00E94CF108091590621
:1037D000A82FB0E0FD01EB5FFB4F808185FF0BC0A0
:1037E000FD01EB59FB4F6081AD59BB4F8C9190E0CF
:1037F00070E00E94371080915906A82FB0E0FD01BB
:10380000EF5FFB4F808183FF0BC0FD01E75EFB4F45
:103810006081A95EBB4F8C9190E070E00E94F10F37
:1038200080915906A82FB0E0FD01EB5FFB4F80812E
:1038300080FF0BC0FD01E35BFB4F6081A55BBB4FCD
:103840008C9190E070E00E949C0F80915906A82F07
:10385000B0E0FD01EF5FFB4F808184FF0BC0FD01F5
:10386000E75DFB4F6081A95DBB4F8C9190E070E0FC
:103870000E945C0F80915906A82FB0E0FD01E75F20
:10388000FB4F808181FF18C080914E06FD01ED57EE
:10389000FB4F813049F4AB57BB4F6C91808190E076
:1038A00070E00E94400E08C0AB57BB4F6C91808106
:1038B00090E070E00E94930E80915906A82FB0E02E
:1038C000FD01ED5FFB4F808187FF0BC0FD01E75BD2
:1038D000FB4F6081A95BBB4F8C9190E070E00E9430
:1038E000830D80915906A82FB0E0FD01EB5FFB4FDF
:1038F000808186FF0BC0FD01E759FB4F6081A9590C
:10390000BB4F8C9190E070E00E94280D089584EAEE
:1039100094E00E948F050E94D3150E94010A089529
:10392000CF93DF93EC0184EA94E00E946604C81709
:10393000D9073CF084EA94E00E945B04892B09F4E7
:103940002397CE01DF91CF910895EF92FF920F93CD
:103950001F93CF93DF930091590610E08AEF90E018
:10396000089F7001099FF00C189FF00C1124C701EB
:103970000E94E60AF801EF5FFB4F882319F080816F
:10398000816002C080818E7F808380915906C82F1C
:10399000D0E0C70102960E94E60AC55FDB4F88832C
:1039A00080915906C82FD0E0C70104960E94E60A0C
:1039B00090E00E94901CC35FDB4F88830091590602
:1039C00010E0C70188569F4F0E94E60AF801EF5F9A
:1039D000FB4F882319F08081806102C080818F7E37
:1039E000808380915906C82FD0E0C70186569F4F2B
:1039F0000E94E60AC95DDB4F888380915906C82F73
:103A0000D0E0C70184569F4F0E94E60A90E00E94D2
:103A1000901CC75DDB4F88830091590610E0C701F9
:103A200006960E94E60AF801EF5FFB4F882319F023
:103A30008081826002C080818D7F80838091590661
:103A4000C82FD0E0C70108960E94E60AC15FDB4F8D
:103A5000888380915906C82FD0E0C7010A960E943A
:103A6000E60A90E00E94901CCF5EDB4F88830091B5
:103A7000590610E0C7010C960E94E60AF801EF5FB4
:103A8000FB4F882319F08081846002C080818B7F86
:103A9000808380915906C82FD0E0C7010E960E94FE
:103AA000E60ACD5EDB4F888380915906C82FD0E0AF
:103AB000C70140960E94E60A90E00E94901CCB5EEF
:103AC000DB4F88830091590610E0C70142960E949F
:103AD000E60AF801EF5FFB4F882319F080818860C8
:103AE00002C08081877F808380915906C82FD0E0F3
:103AF000C70144960E94E60AC95EDB4F8883809125
:103B00005906C82FD0E0C70146960E94E60A90E009
:103B10000E94901CC75EDB4F88830091590610E01D
:103B2000C7014E960E94E60AF801EF5FFB4F88231B
:103B300019F08081806202C080818F7D80838091B6
:103B40005906C82FD0E0C70180960E94E60AC55EDC
:103B5000DB4F888380915906C82FD0E0C701829639
:103B60000E94E60A90E00E94901CC35EDB4F8883AF
:103B70000091590610E0C70184960E94E60AF801F8
:103B8000EF5FFB4F882319F08081806402C0808141
:103B90008F7B808380915906C82FD0E0C70186961D
:103BA0000E94E60AC15EDB4F888380915906C82FC8
:103BB000D0E0C70188960E94E60A90E00E94901C1F
:103BC000CF5DDB4F88830091590610E0C7018A96CC
:103BD0000E94E60AF801EF5FFB4F882319F080810D
:103BE000806802C080818F77808380915906C82FBA
:103BF000D0E0C7018C960E94E60ACD5DDB4F88833A
:103C000080915906C82FD0E0C7018E960E94E60A1F
:103C100090E00E94901CCB5DDB4F88830091590699
:103C200010E0C701C0960E94E60AF801ED5FFB4F65
:103C3000882319F08081816002C080818E7F80831B
:103C400080915906C82FD0E0C701C2960E94E60AAB
:103C5000C55DDB4F888380915906C82FD0E0C7012E
:103C6000C4960E94E60A90E00E94901CC35DDB4F60
:103C700088830091590610E0C701C6960E94E60AA3
:103C8000F801ED5FFB4F882319F08081826002C04C
:103C900080818D7F808380915906C82FD0E0C70135
:103CA000C8960E94E60AC15DDB4F88838091590661
:103CB000C82FD0E0C701CA960E94E60A90E00E9491
:103CC000901CCF5CDB4F88830091590610E0C70140
:103CD000CC960E94E60AF801ED5FFB4F882319F0AD
:103CE0008081846002C080818B7F808380915906AF
:103CF000C82FD0E0C701CE960E94E60ACD5CDB4F0C
:103D0000888380915906C82FD0E0C701805C9F4FFF
:103D10000E94E60A90E00E94901CCB5CDB4F8883F7
:103D20000091590610E0C701885B9F4F0E94E60A88
:103D3000F801ED5FFB4F882319F08081806102C09C
:103D400080818F7E808380915906C82FD0E0C70183
:103D5000865B9F4F0E94E60AC55CDB4F888380919B
:103D60005906C82FD0E0C701845B9F4F0E94E60A26
:103D700090E00E94901CC35CDB4F88830091590641
:103D800010E0C7018E5B9F4F0E94E60AF801ED5FCD
:103D9000FB4F882319F08081886002C08081877F73
:103DA000808380915906C82FD0E0C7018C5B9F4F5C
:103DB0000E94E60AC95CDB4F888380915906C82FB0
:103DC000D0E0C7018A5B9F4F0E94E60A90E00E9404
:103DD000901CC75CDB4F88830091590610E0C70137
:103DE000805B9F4F0E94E60AF801ED5FFB4F88233E
:103DF00019F08081806202C080818F7D80838091F4
:103E00005906C82FD0E0C7018E5A9F4F0E94E60A7C
:103E1000C15CDB4F888380915906C82FD0E0C70171
:103E20008C5A9F4F0E94E60A90E00E94901CCF5B44
:103E3000DB4F88830091590610E0C7018A5A9F4FD3
:103E40000E94E60AF801ED5FFB4F882319F080819C
:103E5000806402C080818F7B808380915906C82F47
:103E6000D0E0C701885A9F4F0E94E60ACD5BDB4F26
:103E7000888380915906C82FD0E0C701865A9F4F8A
:103E80000E94E60A90E00E94901CCB5BDB4F888387
:103E90000091590610E0C70182569F4F0E94E60A22
:103EA000F801ED5FFB4F882319F08081806802C024
:103EB00080818F77808380915906C82FD0E0C70119
:103EC00080569F4F0E94E60AC95BDB4F8883809132
:103ED0005906C82FD0E0C7018E559F4F0E94E60AB1
:103EE00090E00E94901CC75BDB4F888300915906CD
:103EF00010E0C7018E599F4F0E94E60AF801EB5F60
:103F0000FB4F882319F08081816002C080818E7F01
:103F1000808380915906C82FD0E0C7018C599F4FEC
:103F20000E94E60AC55BDB4F888380915906C82F43
:103F3000D0E0C7018A599F4F0E94E60A90E00E9494
:103F4000901CC35BDB4F88830091590610E0C701CA
:103F500082599F4F0E94E60AF801EB5FFB4F8823CE
:103F600019F08081846002C080818B7F8083809182
:103F70005906C82FD0E0C70180599F4F0E94E60A1A
:103F8000C15BDB4F888380915906C82FD0E0C70101
:103F90008E589F4F0E94E60A90E00E94901CCF5AD4
:103FA000DB4F88830091590610E0C70184579F4F6B
:103FB0000E94E60AF801EB5FFB4F882319F080812D
:103FC000806802C080818F77808380915906C82FD6
:103FD000D0E0C70182579F4F0E94E60ACD5ADB4FBF
:103FE000888380915906C82FD0E0C70180579F4F22
:103FF0000E94E60A90E00E94901CCB5ADB4F888317
:104000000091590610E0C7018E569F4F0E94E60AA4
:10401000F801EB5FFB4F882319F08081826002C0BA
:1040200080818D7F808380915906C82FD0E0C701A1
:104030008C569F4F0E94E60AC55ADB4F88838091B9
:104040005906C82FD0E0C7018A569F4F0E94E60A42
:1040500090E00E94901CC35ADB4F88830091590660
:1040600010E0C7018C589F4F0E94E60AF801EB5FF1
:10407000FB4F882319F08081886002C08081877F90
:10408000808380915906C82FD0E0C7018A589F4F7E
:104090000E94E60AC95ADB4F888380915906C82FCF
:1040A000D0E0C70188589F4F0E94E60A90E00E9426
:1040B000901CC75ADB4F88830091590610E0C70156
:1040C00086589F4F0E94E60AF801EB5FFB4F88235A
:1040D00019F08081806102C080818F7E8083809111
:1040E0005906C82FD0E0C70184589F4F0E94E60AA6
:1040F000C15ADB4F888380915906C82FD0E0C70191
:1041000082589F4F0E94E60A90E00E94901CCF596F
:10411000DB4F88830091590610E0C70180589F4FFC
:104120000E94E60AF801EB5FFB4F882319F08081BB
:10413000806202C080818F7D808380915906C82F64
:10414000D0E0C7018E579F4F0E94E60ACD59DB4F42
:10415000888380915906C82FD0E0C7018C579F4FA4
:104160000E94E60A90E00E94901CCB59DB4F8883A6
:104170000091590610E0C7018A579F4F0E94E60A36
:10418000F801EB5FFB4F882319F08081806402C047
:1041900080818F7B808380915906C82FD0E0C70132
:1041A00088579F4F0E94E60AC959DB4F8883809148
:1041B0005906C82FD0E0C70186579F4F0E94E60AD4
:1041C00090E00E94901CC759DB4F888300915906EC
:1041D00010E0C7018C559F4F0E94E60AF801E95F85
:1041E000FB4F882319F08081816002C080818E7F1F
:1041F000808380915906C82FD0E0C7018A559F4F10
:104200000E94E60AC559DB4F888380915906C82F62
:10421000D0E0C70188559F4F0E94E60A90E00E94B7
:10422000901CC359DB4F88830091590610E0C701E9
:1042300080559F4F0E94E60AF801E95FFB4F8823F3
:1042400019F08081846002C080818B7F808380919F
:104250005906C82FD0E0C7018E549F4F0E94E60A2E
:10426000C159DB4F888380915906C82FD0E0C70120
:104270008C549F4F0E94E60A90E00E94901CCF58F9
:10428000DB4F88830091590610E0C7018A549F4F85
:104290000E94E60AF801E95FFB4F882319F080814C
:1042A000886002C08081877F808380915906C82FF3
:1042B000D0E0C70188549F4F0E94E60ACD58DB4FDB
:1042C000888380915906C82FD0E0C70186549F4F3C
:1042D0000E94E60A90E00E94901CCB58DB4F888336
:1042E0000091590610E0C70184549F4F0E94E60ACE
:1042F000F801E95FFB4F882319F08081806102C0DB
:1043000080818F7E808380915906C82FD0E0C701BD
:1043100082549F4F0E94E60AC958DB4F88838091E0
:104320005906C82FD0E0C70180549F4F0E94E60A6B
:1043300090E00E94901CC758DB4F8883009159067B
:1043400010E0C701845A9F4F0E94E60AF801E95F16
:10435000FB4F882319F08081806402C080818F7BAD
:10436000808380915906C82FD0E0C701825A9F4FA1
:104370000E94E60AC558DB4F888380915906C82FF2
:10438000D0E0C701805A9F4F0E94E60A90E00E9449
:10439000901CC358DB4F88830091590610E0C70179
:1043A00080529F4F0E94E60AF801E75FFB4F882387
:1043B00019F08081846002C080818B7F808380912E
:1043C0005906C82FD0E0C7018E519F4F0E94E60AC0
:1043D000C158DB4F888380915906C82FD0E0C701B0
:1043E0008C519F4F0E94E60A90E00E94901CCF578C
:1043F000DB4F88830091590610E0C7018C529F4F14
:104400000E94E60AF801E75FFB4F882319F08081DC
:10441000826002C080818D7F808380915906C82F81
:10442000D0E0C7018A529F4F0E94E60ACD57DB4F6A
:10443000888380915906C82FD0E0C70188529F4FCA
:104440000E94E60A90E00E94901CCB57DB4F8883C5
:10445000DF91CF911F910F91FF90EF9008954F92B0
:104460005F927F928F929F92AF92BF92CF92DF9294
:10447000EF92FF920F931F93DF93CF93CDB7DEB7E9
:10448000C854D0400FB6F894DEBF0FBECDBF04EACB
:1044900014E0C8010E948F05C80166E049E00E944F
:1044A0006A04C8010E94420500D000D0EDB7FEB7F3
:1044B0001283018384EF91E0948383830E94B9295E
:1044C0000F900F900F900F90C8010E94260500D00A
:1044D00000D007E814E0EDB7FEB71283018384EE45
:1044E00091E0948383830E94B92959ED452E51E0D0
:1044F000552EEE24FF24CC24DD240F900F900F9036
:104500000F90702E012F49E0A42EB12CAC0EBD1ED1
:104510004E010894811C911C87E894E00E946D2A4A
:10452000982F8D3031F08D30DCF180538230C0F522
:1045300030C01830A1F59981892F8053823078F5E9
:10454000913311F490E801C090E08A81813309F43D
:10455000905C8B81813309F4905E8C81813309F406
:10456000905F8D81813309F4985F8E81813309F4E6
:104570009C5F8F81813309F49E5F8885813309F4C4
:104580009F5FF501EE0DFF1D90830894E11CF11C67
:1045900006C0F401E10FF11D90831F5F01C010E020
:1045A000F0E4EF16F104C9F484EA94E0B601A50141
:1045B0000E947A040894C11CD11C00D000D0EDB731
:1045C000FEB771820283548243820E94B929EE248D
:1045D000FF240F900F900F900F90FFEFCF16D10494
:1045E00009F00CF499CFC85BDF4F0FB6F894DEBF2B
:1045F0000FBECDBFCF91DF911F910F91FF90EF9034
:10460000DF90CF90BF90AF909F908F907F905F9002
:104610004F900895DF92EF92FF920F931F93DF93D5
:10462000CF93CDB7DEB72A970FB6F894DEBF0FBE93
:10463000CDBF73E0E72EF12CEC0EFD1E63E0D62E0D
:1046400021C40E94633160527E4480409040C8F48F
:104650000E946331695873418040904090F01A3055
:1046600011F01D3031F4809123068F5F8093230673
:1046700002C01092230680912306833011F40E9419
:104680002F22812F69E175E00E94EC06882311F446
:1046900000E0F2C380911D0590911E05A0911F05B9
:1046A000B0912005863E46EA940746E2A4074DE70E
:1046B000B40709F4A0C2873E56EA950756E2A5075B
:1046C0005DE7B50708F0F8C08832EEE59E07E2ED39
:1046D000AE07E4E2BE0709F439C28932FEE59F075E
:1046E000F2EDAF07F4E2BF0708F073C080352FED9D
:1046F00092072DEEA20728E1B20709F479C38135AC
:104700003FED93073DEEA30738E1B30788F584300A
:104710004AE9940747EDA4074EE0B40709F416C22E
:1047200085305AE9950757EDA5075EE0B50780F497
:104730008E3FEBEC9E07E7ECAE07E9E0BE0709F41D
:1047400082C386519A4AA743BB4009F08BC3FEC17E
:10475000823923EA92072CEEA20724E1B20709F47A
:10476000F5C188599C42AA41B64109F07BC3F7C103
:1047700084344BED940740E7A4074DE1B40709F4F6
:1047800062C385345BED950750E7A5075DE1B5078A
:1047900080F48E3CE8E49E07E7E5AE07EAE1BE0759
:1047A00009F429C284579B4EAA47BB4109F05AC35A
:1047B000CDC1823D22EC920722E8A2072EE1B2078A
:1047C00009F4CDC18C5A9A4CA64EB04209F04AC3A6
:1047D0003AC3883546EB94074DEFA4074AE4B40783
:1047E00009F4E8C2893556EB95075DEFA5075AE451
:1047F000B50788F5863EE5ED9E07EAEDAE07E3E3F3
:10480000BE0709F451C1873EF5ED9F07FAEDAF07EA
:10481000F3E3BF0780F48E3729EA92072BE5A2075E
:1048200026E2B20709F49BC182559342A649B642DB
:1048300009F018C36FC2883F4CEA94074EEEA407F4
:1048400044E3B40709F4FFC2865A9E40A241B8442B
:1048500009F008C398C28036EBED9E07EBE3AE0784
:10486000EEE6BE0709F472C18136FBED9F07FBE35C
:10487000AF07FEE6BF0780F4823E25E592072CE9EC
:10488000A20726E6B20709F4A5C28C5E9943A647A3
:10489000BB4609F0E7C2D7C28A3B47EC940741E226
:1048A000A40744E7B40709F4FFC08A57974CA94D01
:1048B000BB4709F0D7C2C7C28C36E8E69E07E3E4DF
:1048C000AE07E2ECBE0709F406C28D36F8E69F0794
:1048D000F3E4AF07F2ECBF0708F073C08A3726EFA6
:1048E000920721EFA2072DE9B20709F484C18B37A3
:1048F00036EF930731EFA3073DE9B30788F58C380E
:1049000045E8940747EAA40748E9B40709F473C1E6
:104910008D3855E8950757EAA50758E9B50780F49B
:104920008634E3E09E07E2ECAE07E5E8BE0709F453
:1049300091C282559A4EA048BA4809F093C206C166
:104940008A362EE2920722E6A20729E9B20709F485
:104950001AC28E579241AA46BB4909F083C2F6C0DB
:104960008A3847EF940747ECA40748EBB40709F4EB
:10497000F6C08B3857EF950757ECA50758EBB507EE
:1049800080F48E3FE6EB9E07E9E2AE07E5EABE075C
:1049900009F431C180529E44A94AB14B09F062C268
:1049A00019C2843A20E092072BE9A2072AEBB2074A
:1049B00009F449C28A5B9448A542BE4B09F052C231
:1049C00009C2843649ED940740EEA40747EDB407C9
:1049D00009F46AC0853659ED950750EEA50757EDE5
:1049E000B50788F58435EDE29E07EFEFAE07E5ECFD
:1049F000BE0709F4ABC08535FDE29F07FFEFAF07A7
:104A0000F5ECBF0780F4803824E7920720E1A20785
:104A100024ECB20709F4A3C086589B43A04AB44CC7
:104A200009F020C2D7C188324FE9940740E0A407BB
:104A300047ECB40709F45FC186599543A840B24DCD
:104A400009F010C267C18E34EDE59E07EEE3AE07B4
:104A5000E3EEBE0709F47AC08F34FDE59F07FEE35D
:104A6000AF07F3EEBF0780F4843727E3920724ED06
:104A7000A2072EEDB20709F4ADC1865B9342A34AAB
:104A8000B24E09F0EFC1B7C0823940E7940746E85B
:104A9000A4074BEFB40709F4D6C1825F9D4EA44230
:104AA000BD4F09F0DFC19FC10E9463316093C8040C
:104AB0007093C9048093CA049093CB04D092C70426
:104AC00089E195E060E170E00E94C0080E946B34CB
:104AD0007093CD046093CC0489E195E064E170E0CB
:104AE0000E94C0080E946B347093CF046093CE0480
:104AF00089E195E068E170E00E94C0080E946B3493
:104B00008B017093D1046093D0046091D2047091B2
:104B1000D3048091D4049091D50420E030E040E0AB
:104B200050E00E94FC33882379F4B801882777FD90
:104B30008095982F0E949E346093D6047093D7047A
:104B40008093D8049093D90401E08DC1809123050E
:104B50008093DA04809124058093DB0483C189E18A
:104B600095E060E070E00E94C00820E030E048EC92
:104B700052E40E94D1350E946B347093DD0460933F
:104B8000DC04693C710520F01092DD041092DC0415
:104B900080913D0590913E059093DF048093DE0463
:104BA00080913F05909140059093E1048093E0044B
:104BB00080914305909144059093A4028093A302B1
:104BC00080914705909148059093A6028093A50295
:104BD0008091490590914A059093A8028093A7027D
:104BE00080914B0590914C059A8389839093AA02FA
:104BF0008093A90237C160912305709124058091AB
:104C00002505909126050E949E3420E836E948E16A
:104C10005BE40E9403346093D2047093D3048093C6
:104C2000D4049093D5046091270570912805809154
:104C3000290590912A05D7016C9311967C931197C1
:104C400012968C93129713969C930E949E3420E8A0
:104C500036E948E15BE40E9403346093E204709318
:104C6000E3048093E4049093E504809148058093E5
:104C7000E6048091470584300CF083E08093E704DC
:104C800089E195E060E170E00E94C0086093D6047D
:104C90007093D7048093D8049093D90489E195E068
:104CA00068E070E00E94C0086093E8047093E90433
:104CB0008093EA049093EB0489E195E064E170E06D
:104CC0000E94C0086093EC047093ED048093EE049E
:104CD0009093EF04C7C089E195E068E070E00E941E
:104CE000C00890586093F0047093F1048093F2042C
:104CF0009093F304B7C089E195E060E070E00E9412
:104D0000C0086093F4047093F5048093F6049093C4
:104D1000F704A8C089E195E060E070E00E94C00857
:104D20006093F8047093F9048093FA049093FB0461
:104D300089E195E064E070E00E94C00820E030E086
:104D400048EC52E40E94D1350E946B347093FD040C
:104D50006093FC0489E195E064E170E00E94C00882
:104D60000E946B347093FF046093FE0489E195E028
:104D700068E170E00E94C0080E946B3470930105E6
:104D8000609300056FC089E195E064E070E00E94E7
:104D9000C0080E946B34882777FD8095982F0E9469
:104DA0009E346093020570930305809304059093ED
:104DB000050558C089E195E068E070E00E94C008F0
:104DC0000E946B34709561957F4F709307056093D7
:104DD000060548C08091830580930805809184056D
:104DE000809309053FC08091230580930A053AC04E
:104DF00089E195E060E070E00E94C00860930B05D7
:104E000070930C0580930D0590930E0589E195E054
:104E100064E070E00E94C00860930F057093100575
:104E2000809311059093120589E195E068E070E0A8
:104E30000E94C008609313057093140580931505B4
:104E4000909316050FC080912F05809317058091D0
:104E5000340506C080913005809317058091350593
:104E60008093180500E080911A05823229F489E1C7
:104E700095E063E20E94D8098EEB90E00E94CA316F
:104E8000002331F587E894E00E943D2A18161906A0
:104E9000F4F487E894E00E946D2A182F8091C704EB
:104EA000882309F0EECBCDCB1092C70401E0802F10
:104EB00090E02A960FB6F894DEBF0FBECDBFCF911B
:104EC000DF911F910F91FF90EF90DF90089500E028
:104ED0002091C8043091C9044091CA045091CB0478
:104EE000205F384D4F4F5F4F2F83388749875A8750
:104EF0000E9463312F81388549855A8526173707E7
:104F00004807590788F2D3CF1F93CF93DF9385E0EB
:104F100090E06CE070E00E94091668EE73E080E0BB
:104F200090E00E94713187E894E00E94BA2AC0E0C4
:104F3000D0E010E0CE016DE171E00E940B37892BCB
:104F4000A9F41F5E84EA94E0612F4CE00E946A0499
:104F500084EA94E00E94420584EA94E06EEE0E94A6
:104F6000720584EA94E00E942605105161E070E029
:104F700080E090E00E947131219687E0C13DD80722
:104F8000C9F6DF91CF911F91089586E061E00E94FC
:104F9000A83208950F931F9386E061E00E94693262
:104FA00007E814E0C80140E051EE60E070E00E94C4
:104FB000DB291093A2060093A1060E94C52784EA6C
:104FC00094E00E94C8050E94871C64EF71E080E0B5
:104FD00090E00E94713183EF93E00E94E60A8130F5
:104FE00011F00E94F70C0E94570A1092590607C050
:104FF0000E94A51C809159068F5F8093590680916D
:1050000059068230A8F3109259060E94842786EB35
:1050100094E069E979E224E630E040E050E000E025
:105020000E948E3084EA94E00E948F0586EB94E023
:105030000E94F4301F910F9108952F923F924F924A
:105040005F926F927F928F929F92AF92BF92CF9218
:10505000DF92EF92FF920F931F93DF93CF9300D0D5
:1050600000D0CDB7DEB780915506882309F4E1C0A2
:10507000E0907A06F0907B0600917C0610917D0608
:10508000C801B7019F7725E33AEF4EE85CE30E9441
:10509000D1350E94003469837A838B839C83C80155
:1050A000B7012091D2043091D3044091D40450919F
:1050B000D5040E9435331B012C019F7720EC3BE681
:1050C00049ED57E40E94D1355B016C0160917E0689
:1050D00070917F0680918006909181062091E20474
:1050E0003091E3044091E4045091E5040E9435338B
:1050F0003B014C019F7720EC3BE649ED57E40E94D1
:10510000D13529813A814B815C810E94D1357B0167
:105110008C01C601B501A60195010E94D1355B0144
:105120006C01C801B701A80197010E94D1359B010C
:10513000AC01C601B5010E9436330E9458360E9468
:105140006B34609348067093490680934A069093A7
:105150004B0660E070E080E89FE329813A814B8153
:105160005C810E9403349B01AC01C201B1010E9429
:10517000D13597FA909497F89094A40193010E94E6
:10518000A93320EE3EE245E652E40E94D13520E00C
:1051900030E044EB52E40E9436330E946B349B01B2
:1051A000AC0197FF04C028593E4F4F4F5F4FCA01D3
:1051B000B901645B70408040904097FF06C0CA010F
:1051C000B9016C547F4F8F4F9F4F0E949E342091A6
:1051D000D6043091D7044091D8045091D9040E944C
:1051E00035330E946B3497FF04C068597E4F8F4F50
:1051F0009F4F0E949E3420E030E044EB53E40E9435
:10520000033420E030E040E851E40E94D1350E94B0
:10521000343620E030E040E85FE30E9436330E94FD
:10522000703460934706613108F46CC010924706F1
:1052300069C08091E704823008F464C08091E6047C
:10524000853008F45FC0A09082068DE18A1508F4CD
:1052500059C0E090E804F090E9040091EA0410914C
:10526000EB0460918306709184068091850690918D
:105270008606A80197010E9435339F7720E030E031
:1052800040E05FE30E94C63518165CF41092820677
:10529000E0928306F09284060093850610938606BA
:1052A00031C08A2D8F5F809382068E3159F58091AF
:1052B000D2049091D304A091D404B091D5048093EA
:1052C0007A0690937B06A0937C06B0937D0680912E
:1052D000E2049091E304A091E404B091E50480938A
:1052E0007E0690937F06A0938006B0938106E0929D
:1052F0008706F09288060093890610938A0681E05B
:10530000809355060F900F900F900F90CF91DF91E3
:105310001F910F91FF90EF90DF90CF90BF90AF90D3
:105320009F908F907F906F905F904F903F902F90C5
:10533000089580910A058093AB021092AC020E94FE
:1053400049080E94EC0A84EA94E00E941D280E9409
:10535000561A08950E940A23892B19F00E94992950
:10536000089586EB94E00E94DC3008958FEF9FE76C
:105370000895DF93CF93CDB7DEB7FE0139968D81C7
:105380009E8161E04F8158859F010E945A2CCF91E8
:10539000DF910895DF93CF93CDB7DEB7FE01399645
:1053A0008D819E8160E04F8158859F010E945A2C1B
:1053B000CF91DF9108950F931F93DC01ED91FC9144
:1053C0000288F389E02D20E030E000E010E009954C
:1053D0001F910F9108958F92AF92CF92EF92FF920B
:1053E0000F931F93DF93CF93CDB7DEB7FC011382EA
:1053F000128288EE93E0A0E0B0E084839583A683D8
:10540000B78389EE93E091838083558744873787FC
:105410002687118B008BF38AE28AC48AA58A868A42
:1054200070E0CB0123E0880F991F2A95E1F79C01DA
:105430002157394F308F278B8956994F928F818F03
:1054400081E090E002C0880F991F6A95E2F72091F1
:105450009F06282B20939F06CF0140E051EE60E08D
:1054600070E00E94DB29CF91DF911F910F91FF9097
:10547000EF90CF90AF908F900895FC01838D88239B
:1054800019F42FEF3FEF0DC00788F08DE02D20813C
:10549000318182819381281B390B84819581282356
:1054A0003923C9010895FC01838D882319F42FEF56
:1054B0003FEF11C0018CF28DE02D2081318182817E
:1054C0009381281B390B2095309584819581282361
:1054D00039232F5F3F4FC9010895FC01838D882335
:1054E00061F0A789B08D2D913C91119712968D9105
:1054F0009C9113972817390721F44FEF5FEFCA01EA
:10550000089512968D919C9113971696ED91FC91AA
:105510001797E80FF91F408112968D919C91139770
:10552000019614962D913C911597822393231396FF
:105530009C938E93129750E0E2CFFC01838D8823D9
:1055400051F00788F08DE02D208131818281938197
:105550002817390721F42FEF3FEFC9010895828101
:1055600093810680F781E02DE80FF91F8081282FB5
:1055700030E0F3CFDC015796ED91FC915897828192
:105580009381918380835996ED91FC915A97808104
:105590009181938382830895DC015B968C915B9764
:1055A0008823A9F15996ED91FC915A972081318178
:1055B0002F5F3F4F84819581282339235C968C91FE
:1055C0005C97882329F08281938128173907F9F0A5
:1055D0008281938128173907D9F3808191810680D0
:1055E000F781E02DE80FF91F60835996ED91FC914A
:1055F0005A97318320835296ED91FC915397808185
:1056000056969C91892B808321E030E002C020E0F7
:1056100030E0C9010895CF93DF93EC011B821A8219
:105620008A819B81998388831D821C828E819F81C0
:10563000009721F00E94BC031F821E82DF91CF9150
:1056400008950F931F938C01DC015296ED91FC910C
:105650005397208156968C91569755969C915597C5
:10566000892B80958223808357968D919C915897A2
:105670000E940B2BF801818D928D0E940B2BD8017B
:105680005B961C921F910F9108950F931F93CF93D8
:10569000DF938C01FC0113821282828193819183BA
:1056A000808341E0A1E0B0E001C04F5FFD01042E26
:1056B00002C0EE0FFF1F0A94E2F79B0182E0613007
:1056C000780710F020E032E0E217F30770F3C1E052
:1056D000D0E002C0CC0FDD1F4A95E2F72197F80118
:1056E000268137812115310541F0848195818C1700
:1056F0009D0789F0C9010E94BC03F801D583C483CA
:10570000CE0101960E9412039C01F80197838683C3
:1057100080E0232B09F081E0DF91CF911F910F9161
:105720000895AF92BF92CF92DF92EF92FF920F93C4
:105730001F93CF93DF937C015A016B01E901DC01D8
:105740005B968C915B978823F1F02115310539F434
:105750005796ED91FC915897C481D58121960115FA
:10576000110549F4D7015996ED91FC915A9704819E
:1057700015810F5F1F4FD701ED91FC910088F189D2
:10578000E02DC7010995F7018789908D209711F4C5
:10579000C0E8D0E0BE010E94452B882381F0D701EC
:1057A00059968D919C915A970115110511F400E1BC
:1057B00010E0B8010E94452B882309F04DC0D701A5
:1057C000ED91FC910088F189E02DC701099567C032
:1057D000D7015096ED91FC915197B0E0AB16B1EE28
:1057E000BB06B0E0CB06B0E0DB0609F454C081E0B4
:1057F00090E0D70154960C9002C0880F991F0A942C
:10580000E2F7808360E079E08DE390E0A601950106
:105810000E9440372150304040405040CA01B901F9
:1058200022E030E040E050E00E944037D7011C9673
:10583000ED91FC911D9730831E96ED91FC911F9781
:105840002083D7015296ED91FC9153978081559614
:105850009C91892B808323C0D7015996ED91FC91AF
:105860005A97138212828281938191838083579603
:10587000ED91FC91589713821282828193819183DA
:10588000808381E05B968C931A141B041C041D0416
:105890000CF49ECFD6CF108220E130E0C7CFDF914D
:1058A000CF911F910F91FF90EF90DF90CF90BF901D
:1058B000AF9008952F923F924F925F926F927F9296
:1058C0008F929F92AF92BF92CF92DF92EF92FF9210
:1058D0000F931F93DF93CF93CDB7DEB764970FB6C7
:1058E000F894DEBF0FBECDBF3C01688B5A8B498B4D
:1058F00069011C01AE014F5F5F4F5C8B4B8BE989E7
:10590000FA89488940FD659140FF6191FA8BE98BE6
:10591000662309F4D7C3653249F440FD859140FF01
:105920008191FA8BE98B8532B1F40CC06A3051F465
:10593000D301ED91FC910190F081E02DC1016DE06A
:1059400009956AE0D301ED91FC910190F081E02D81
:10595000C1010995D4CF982F10E0882499241032E2
:10596000B0F49B3269F09C3228F4903251F09332BB
:1059700071F40BC09D3239F0903349F4116028C0A6
:105980001260146025C0186023C0106121C017FD8B
:105990002BC0892F80538A3078F416FF06C0BAE0F6
:1059A0009B9E902C1124980E13C0EAE08E9E802CB2
:1059B0001124880E10620CC09E3221F416FD82C3A1
:1059C000106406C09C3611F4106802C0983661F469
:1059D000E989FA89488940FD959140FF9191FA8BB8
:1059E000E98B992309F0BBCF892F8554833020F4AC
:1059F000812F8061905E07C0892F8556833008F023
:105A0000E6C1812F8F7E86FD02C076E0972E6FE380
:105A1000F62EF822953619F450E4F52A07C096368A
:105A200019F480E8F82A02C091109A94F7FE0BC08E
:105A30009BE3991520F427E05CE3B52E0DC0B92C4B
:105A4000B39427E009C0A7E0A91520F447E0942EFD
:105A500027E001C0292DBB24F6013496FD87EC8791
:105A6000D6016D917D918D919C91AE014F5F5F4FFD
:105A70000B2D0E943A026C010981E02FF0E0FF87B4
:105A8000EE8700FF05C0FE85F3FD02C01DE209C0E0
:105A9000F1FE02C01BE205C0F2FC02C010E001C032
:105AA00010E28E859F858C709070892B09F444C01C
:105AB000112311F483E001C084E0881510F08824DC
:105AC0000EC0881AF3FC0BC0D301ED91FC9101903C
:105AD000F081E02DC10160E209958A94A9F71123B4
:105AE00049F0D301ED91FC910190F081E02DC101CD
:105AF000612F0995BE85B3FF03C00DEF12E012C000
:105B000001E013E00FC0E114F10409F06052D30189
:105B1000ED91FC910190F081E02DC10109950F5F9D
:105B20001F4F05C0EF2CFF24B0E1EB22FF24F8014A
:105B30006491662341F748C1F7FE13C0BC0CFE8593
:105B4000F4FF04C08A81813309F4BA941B141CF059
:105B5000BB24B3942DC048E04B1550F538E0B32E6C
:105B600027C0F6FC25C0892D90E08C159D054CF0D2
:105B70005CEFC5165FEFD50624F080E8F82A01C077
:105B80009A94992049F0E2E0F0E0EC0FFD1FE90D56
:105B9000F11D80818033A1F3F7FE0AC0B92CB394C4
:105BA000892D90E0C816D90614F0992401C09C18DC
:105BB000F7FC03C025E030E009C01C141D041CF0F4
:105BC00021E030E003C096012F5F3F4F112311F019
:105BD0002F5F3F4F992029F0892D90E00196280FE3
:105BE000391F882D90E02817390714F0882401C048
:105BF000821A4F2C5524C20189709070892B59F05C
:105C00000CC0D301ED91FC910190F081E02DC10118
:105C100060E209958A948820A1F7112349F0D30105
:105C2000ED91FC910190F081E02DC101612F09956A
:105C300043FE0BC00CC0D301ED91FC910190F081AB
:105C4000E02DC10160E309958A948820A1F7F7FE51
:105C500051C08601D7FE02C000E010E07601089432
:105C6000E11CF11CE01AF10AE1E0F0E0EC0FFD1F8D
:105C7000EE0EFF1E26014B185108892D90E0AA2434
:105C8000BB24A81AB90AFFEF0F3F1F0749F4D3013D
:105C9000ED91FC910190F081E02DC1016EE209953A
:105CA000C016D10634F0401651061CF4F70160818D
:105CB00001C060E3015010400894E11CF11C0A157A
:105CC0001B054CF0D301ED91FC910190F081E02D8A
:105CD000C1010995D8CF0C151D0541F48A81863381
:105CE00020F4853319F4BE85B4FF61E3D301ED914F
:105CF000FC9165C06A81613309F00F7ED301ED919B
:105D0000FC910190F081E02DC10109959920E1F00D
:105D1000D301ED91FC910190F081E02DC1016EE283
:105D2000099512E0E1E0F0E0EC0FFD1FE10FF11D3D
:105D300060811F5FD301ED91FC910190F081E02D16
:105D4000C10109959A9471F7D301ED91FC910190ED
:105D5000F081E02D44FC02C065E601C065E4C101AC
:105D60000995D7FC05C0C114D10441F404FF06C055
:105D7000D094C194D108D3946DE201C06BE2D301F9
:105D8000ED91FC910190F081E02DC101099560E356
:105D900005C06F5FE6EFFFEFCE0EDF1EFAE0CF1615
:105DA000D104BCF7D301ED91FC910190F081E02D7D
:105DB000C1010995D301ED91FC916C2D605D0190BD
:105DC000F081E02DC1010995CC84DD8478C1933642
:105DD00031F0933799F0933509F061C023C0F60193
:105DE000808189835E010894A11CB11C42E050E0CF
:105DF000C40ED51E21E0E22EF12C12C0D601AD90CA
:105E0000BC9016FD03C06FEF7FEF02C0692D70E0FC
:105E1000E2E0F0E0CE0EDF1EC5010E941F047C010F
:105E20001F7713C0D601AD90BC9016FD03C06FEF75
:105E30007FEF02C0692D70E0E2E0F0E0CE0EDF1EE1
:105E4000C5010E9414047C01106813FF0BC023C01D
:105E5000D301ED91FC910190F081E02DC10160E250
:105E600009958A94882D90E0E816F90688F313C006
:105E7000F50117FD659117FF61915F01D301ED9168
:105E8000FC910190F081E02DC101099581108A9467
:105E90000894E108F108E114F10451F710C19436B7
:105EA00011F0993699F517FF0AC0F601208131816A
:105EB0004281538184E090E0C80ED91E0CC0D60107
:105EC0008D919C919C01442737FD4095542FE2E031
:105ED000F0E0CE0EDF1E9FE6F92EF12257FF09C03B
:105EE00050954095309521953F4F4F4F5F4FF0E8CB
:105EF000FF2ACA01B901AE014F5F5F4F2AE030E0CF
:105F00000E94DC01E82E4B89E41A41C0953721F448
:105F10001F7E2AE030E01CC0197F9F3661F0903769
:105F200020F4983509F0CEC00FC0903739F098377B
:105F300009F0C8C004C028E030E00AC0106114FDB8
:105F4000146020E130E004C014FD166020E132E06E
:105F500017FF08C0D6016D917D918D919C91E4E071
:105F6000F0E008C0D6018D919C91BC0180E090E0EA
:105F7000E2E0F0E0CE0EDF1EAE014F5F5F4F0E9409
:105F8000DC01E82EFB89EF1A8FE7F82EF122F6FEEE
:105F90000BC04EEFF422E91438F4F4FE07C0F2FC13
:105FA00005C05FEEF52202C01E2D01C0192DF4FEC2
:105FB0000DC0FE01EE0DF11D8081803319F489EED4
:105FC000F82208C01F5FF2FE05C003C08F2D86783F
:105FD00009F01F5F0F2DF3FC18C0F0FE13C0181559
:105FE00010F09E2C0FC09E2C980C911A182D0AC0F0
:105FF000D301ED91FC910190F081E02DC10160E2AF
:1060000009951F5F1815A0F304C0181510F4811A24
:1060100001C0882404FF17C0D301ED91FC910190C9
:10602000F081E02DC10160E3099502FF29C0D30191
:10603000ED91FC910190F081E02D01FD02C068E737
:1060400012C068E510C0802F8678D1F001FF02C031
:106050006BE201C060E2F7FC6DE2D301ED91FC91CF
:106060000190F081E02DC10109950AC0D301ED91A5
:10607000FC910190F081E02DC10160E309959A94B3
:10608000E914A0F3EA94D301ED91FC91A1E0B0E012
:10609000AC0FBD1FAE0DB11D0190F081E02DC1010F
:1060A0006C910995EE2071F70AC0D301ED91FC9136
:1060B0000190F081E02DC10160E209958A94882069
:1060C000A1F71DCC64960FB6F894DEBF0FBECDBF0E
:1060D000CF91DF911F910F91FF90EF90DF90CF90C4
:1060E000BF90AF909F908F907F906F905F904F90F8
:1060F0003F902F900895F999FECF72BD61BDF89A37
:1061000080B50895F999FECF1FBA72BD61BD40BD3B
:106110000FB6F894FA9AF99A0FBE08950F93FC01FE
:106120006115710511F480E011C02183328343832E
:106130005483728761870170000F000F000F808108
:10614000877F802B82608B7F808381E00F91089511
:10615000CF93DF93EC010E9463319B01AC018D81F1
:106160009E81AF81B885281739074A075B0728F455
:10617000888184FD02C060E00DC089819A81AB8175
:10618000BC81820F931FA41FB51F8D839E83AF8395
:10619000B88761E0222757FD2395332744275527E9
:1061A000922F91709295907F88818F7E892B888322
:1061B000862FDF91CF910895CF93DF93EC018881F3
:1061C00082FF0FC0CE010E94A830882351F0E985DC
:1061D000FA85309709F00995888183FF02C08B7F8B
:1061E0008883DF91CF910895CF93DF93EC01898568
:1061F0009A85892BE1F089819A81AB81BC810097D6
:10620000A105B105A1F00E94633129813A814B813A
:106210005C81260F371F481F591F2D833E834F83F4
:106220005887888184608F7E888381E001C080E008
:10623000DF91CF9108951F920F920FB60F92112404
:106240002F933F938F939F93AF93BF938091A70614
:106250009091A806A091A906B091AA063091AB062C
:106260000196A11DB11D232F2D5F2D3720F02D5735
:106270000196A11DB11D2093AB068093A7069093B4
:10628000A806A093A906B093AA068091A3069091B0
:10629000A406A091A506B091A6060196A11DB11D68
:1062A0008093A3069093A406A093A506B093A60698
:1062B000BF91AF919F918F913F912F910F900FBE02
:1062C0000F901F9018958FB7F8942091A7063091E2
:1062D000A8064091A9065091AA068FBFB901CA012C
:1062E00008959B01AC017FB7F8948091A30690912B
:1062F000A406A091A506B091A60666B5A89B05C008
:106300006F3F19F00196A11DB11D7FBFBA2FA92FB4
:10631000982F8827860F911DA11DB11D62E0880F5F
:10632000991FAA1FBB1F6A95D1F7BC012DC0FFB7EB
:10633000F8948091A3069091A406A091A506B0912F
:10634000A606E6B5A89B05C0EF3F19F00196A11D72
:10635000B11DFFBFBA2FA92F982F88278E0F911D2F
:10636000A11DB11DE2E0880F991FAA1FBB1FEA956E
:10637000D1F7861B970B885E9340C8F221503040BE
:106380004040504068517C4F211531054105510571
:1063900071F60895019739F0880F991F880F991F9A
:1063A00002970197F1F70895789484B5826084BDCF
:1063B00084B5816084BD85B5826085BD85B5816009
:1063C00085BDEEE6F0E0808181608083E1E8F0E069
:1063D0001082808182608083808181608083E0E898
:1063E000F0E0808181608083E1EBF0E08081846077
:1063F0008083E0EBF0E0808181608083EAE7F0E079
:1064000080818460808380818260808380818160DC
:1064100080838081806880831092C10008951F92DC
:106420000F920FB60F9211242F933F934F935F93C8
:106430006F937F938F939F93AF93BF93EF93FF934C
:106440008091AC069091AD06892B29F0E091AC06C5
:10645000F091AD060995FF91EF91BF91AF919F919A
:106460008F917F916F915F914F913F912F910F90FD
:106470000FBE0F901F9018951F920F920FB60F929C
:1064800011242F933F934F935F936F937F938F9339
:106490009F93AF93BF93EF93FF938091AE0690913C
:1064A000AF06892B29F0E091AE06F091AF06099571
:1064B000FF91EF91BF91AF919F918F917F916F91DC
:1064C0005F914F913F912F910F900FBE0F901F90B2
:1064D0001895CF93DF93482F50E0CA01895C9C4FF9
:1064E000FC0134914D5D5C4FFA018491882369F180
:1064F00090E0880F991FFC01EB5FFC4FA591B491D0
:10650000FC01E15FFC4FC591D491662351F42FB794
:10651000F8948C91932F909589238C93888189236B
:106520000BC0623061F42FB7F8948C91932F909543
:1065300089238C938881832B88832FBF06C09FB7C4
:10654000F8948C91832B8C939FBFDF91CF9108950A
:10655000482F50E0CA01855B9C4FFC012491CA0181
:10656000895C9C4FFC0194914D5D5C4FFA01349124
:10657000332309F440C0222351F1233071F0243039
:1065800028F42130A1F0223011F514C02630B1F0EA
:106590002730C1F02430D9F404C0809180008F7777
:1065A00003C0809180008F7D8093800010C084B5EF
:1065B0008F7702C084B58F7D84BD09C08091B00003
:1065C0008F7703C08091B0008F7D8093B000E32F60
:1065D000F0E0EE0FFF1FE15FFC4FA591B4912FB7E4
:1065E000F894662321F48C919095892302C08C91B4
:1065F000892B8C932FBF0895CF92DF92EF92FF9259
:106600000F931F93CF93DF937C016B018A01C0E04E
:10661000D0E00FC0D6016D916D01D701ED91FC91D5
:106620000190F081E02DC7010995C80FD91F0150D5
:1066300010400115110571F7CE01DF91CF911F9127
:106640000F91FF90EF90DF90CF900895CF93DF935D
:106650000E94D4310E94CA27C0E0D0E00E94AA293B
:106660002097E1F30E940000F9CF5058BB27AA27DA
:106670000ED041C201D230F006D220F031F49F3F5B
:1066800011F41EF4C0C10EF4E095E7FBB6C1E92F8A
:1066900054D280F3BA17620773078407950718F07E
:1066A00071F49EF56CC20EF4E0950B2EBA2FA02D5E
:1066B0000B01B90190010C01CA01A0011124FF27AF
:1066C000591B99F0593F50F4503E68F11A16F040AA
:1066D000A22F232F342F4427585FF3CF46953795A9
:1066E0002795A795F0405395C9F77EF41F16BA0B6E
:1066F000620B730B840BBAF09150A1F0FF0FBB1F1C
:10670000661F771F881FC2F70EC0BA0F621F731F64
:10671000841F48F4879577956795B795F7959E3FC1
:1067200008F0B3CF9395880F08F09927EE0F97954F
:1067300087950895A1D158F080E891E009F49EEF83
:10674000A2D128F040E851E059F45EEF09C05BC1E6
:1067500016C2E92FE078F1D168F3092E052AC1F3BA
:10676000261737074807590738F00E2E07F8E02597
:1067700069F0E025E0640AC0EF6307F8009407FAC7
:10678000DB01B9019D01DC01CA01AD01EF934AD0E3
:10679000B2D10AD05F91552331F02BED3FE049E4AF
:1067A00050FD49EC63CF0895DF93DD27B92FBF7704
:1067B00040E85FE31616170648075B0710F4D92F69
:1067C000E9D19F938F937F936F93BCD2E8E6F0E07B
:1067D0001DD191D12F913F914F915F91EED1DD234A
:1067E00049F09058A2EA2AED3FE049EC5FE3D07807
:1067F0005D274DDFDF917FC1DCD008F481E0089593
:106800004AD1E39589C10CD076C13DD140F034D155
:1068100030F021F45F3F19F0F0C05111B1C1F3C065
:106820008CD198F39923C9F35523B1F3951B550BDC
:10683000BB27AA2762177307840738F09F5F5F4F53
:10684000220F331F441FAA1FA9F333D00E2E3AF094
:10685000E0E830D091505040E695001CCAF729D0AE
:10686000FE2F27D0660F771F881FBB1F26173707FD
:106870004807AB07B0E809F0BB0B802DBF01FF272D
:1068800093585F4F2AF09E3F510568F0B6C078C11B
:106890005F3FECF3983EDCF3869577956795B79567
:1068A000F7959F5FC9F7880F911D9695879597F982
:1068B0000895E1E0660F771F881FBB1F62177307FB
:1068C0008407BA0720F0621B730B840BBA0BEE1F10
:1068D00088F7E095089504D06894B11151C10895E6
:1068E00034D188F09F5790F0B92F9927B751A0F075
:1068F000D1F0660F771F881F991F1AF0BA95C9F754
:1069000012C0B13081F03BD1B1E0089538C1672F9A
:10691000782F8827B85F39F0B93FCCF38695779503
:106920006795B395D9F73EF49095809570956195EC
:106930007F4F8F4F9F4F0895E89409C097FB3EF417
:1069400090958095709561957F4F8F4F9F4F9923BC
:10695000A9F0F92F96E9BB279395F695879577953A
:106960006795B795F111F8CFFAF4BB0F11F460FFFA
:106970001BC06F5F7F4F8F4F9F4F16C0882311F052
:1069800096E911C0772321F09EE8872F762F05C066
:10699000662371F096E8862F70E060E02AF09A9501
:1069A000660F771F881FDAF7880F9695879597F9F6
:1069B0000895990F0008550FAA0BE0E8FEEF161690
:1069C0001706E807F907C0F012161306E407F507E3
:1069D00098F0621B730B840B950B39F40A2661F057
:1069E000232B242B252B21F408950A2609F4A140FA
:1069F000A6958FEF811D811D089597F99F6780E807
:106A000070E060E008959FEF80EC0895DF93CF93EE
:106A10001F930F93FF92EF92DF927B018C0168949A
:106A200005C0DA2EEF01C9D0FE01E894A5912591A9
:106A3000359145915591AEF3EF0129DEFE019701A5
:106A4000A801DA9479F7DF90EF90FF900F911F91F2
:106A5000CF91DF9108959F938F937F936F93FF93CF
:106A6000EF939B01AC019DD0EF91FF91CFDF2F9170
:106A70003F914F915F9195C000240A941616170616
:106A800018060906089500240A941216130614061F
:106A900005060895B8CF59D0E8F3E894EFEFBB2787
:106AA0003FE048EC5FE76B3D73078407950708F10B
:106AB000FF279F57B25A6A4D7F40894CF04032F40D
:106AC000BE556542704F8643FF4F0894EE1F9150AC
:106AD00030F0BB0F661F771F881FFF1FEBCF9EE7AD
:106AE000882332F0BB0F661F771F881F9A95C1F766
:106AF0009395E09565C1092E0394000C11F4882349
:106B000052F0BB0F40F4BF2B11F460FF04C06F5F65
:106B10007F4F8F4F9F4F0895EF93E0FF06C0A2EA8B
:106B20002AED3FE049EC5FEBB2DDE5DF0F90039427
:106B300001FC9058E5E9F0E08ECF57FD9058440FE6
:106B4000551F59F05F3F71F04795880F97FB991FCC
:106B500061F09F3F79F08795089512161306140689
:106B6000551FF2CF4695F1DF08C016161706180616
:106B7000991FF1CF86957105610508940895E894F1
:106B8000BB2766277727CB0197F9089512DF08F412
:106B90008FEF08959B01AC0160E070E080E89FE317
:106BA00032CE0BD0A8CF68DF28F06DDF18F0952328
:106BB00009F023CF28CF1124E3CFBFDFA0F3959FA7
:106BC000D1F3950F50E0551F629FF001729FBB27D4
:106BD000F00DB11D639FAA27F00DB11DAA1F649F80
:106BE0006627B00DA11D661F829F2227B00DA11D33
:106BF000621F739FB00DA11D621F839FA00D611DB9
:106C0000221F749F3327A00D611D231F849F600DD9
:106C1000211D822F762F6A2F11249F5750408AF012
:106C2000E1F088234AF0EE0FFF1FBB1F661F771F9E
:106C3000881F91505040A9F79E3F510570F0DDCE5E
:106C40009FCF5F3FECF3983EDCF386957795679591
:106C5000B795F795E7959F5FC1F7FE2B880F911DBC
:106C60009695879597F9089570DFE0F09E37D8F0F4
:106C70009639B8F49E3848F4672F782F8827985FA4
:106C8000F9CF86957795679593959539D0F3B62F7B
:106C9000B1706B0F711D811D20F4879577956795F5
:106CA000939573C08DC06CCF11F40EF4ACCE88C038
:106CB0004CDFD0F39923D9F3CEF39F57550B87FFC1
:106CC0008FD056959795B0E020F4660F771F881FF8
:106CD000BB1F1F930F9300249001A0018001F001BE
:106CE000A0E80E0F1F1F0A1E511D601B710B8009AB
:106CF000B50B48F4600F711F801DB51F0E1B1F0BD5
:106D00000A0A510907C02E0F3F1F4A1F0E0F1F1FEF
:106D10000A1E511D660F771F881FBB1FA695F7958A
:106D2000E795F8F60617170708065B07211D311DC2
:106D3000411D0F911F91B901842F9158880F96958D
:106D4000879508959B01AC012CCFDF93D92FA3DE4B
:106D5000E695D7952AED3FE049E45FE3B33A620751
:106D6000730784079507D7952AF0A2EA49EC906843
:106D70008EDCC1DEE3EBF0E06EDEDD0F0BF00ADF50
:106D8000DD0F0BF49058DF910895882371F4772379
:106D900021F09850872B762F07C0662311F499278E
:106DA0000DC09051862B70E060E02AF09A95660F36
:106DB000771F881FDAF7880F9695879597F90895BA
:106DC0009F3F49F0915028F4869577956795B79540
:106DD0009F5F80389F4F880F9695879597F9089504
:106DE00091505040660F771F881FD2F70895AA1B55
:106DF000BB1B51E107C0AA1FBB1FA617B70710F0A6
:106E0000A61BB70B881F991F5A95A9F780959095D7
:106E1000BC01CD01089597FB092E07260AD077FD06
:106E200004D0E5DF06D000201AF4709561957F4FFD
:106E30000895F6F7909581959F4F0895A1E21A2E37
:106E4000AA1BBB1BFD010DC0AA1FBB1FEE1FFF1F0E
:106E5000A217B307E407F50720F0A21BB30BE40B5E
:106E6000F50B661F771F881F991F1A9469F76095A5
:106E70007095809590959B01AC01BD01CF0108955F
:106E800097FB092E05260ED057FD04D0D7DF0AD078
:106E9000001C38F450954095309521953F4F4F4F49
:106EA0005F4F0895F6F790958095709561957F4FA7
:106EB0008F4F9F4F0895EE0FFF1F0590F491E02D27
:066EC0000994F894FFCFD5
:106EC600256300256325630025632532692563252F
:106ED6003032697C256325326925632530326900A5
:106EE60025632532692563253032690025352E3024
:106EF60066256300256325312E35662563002563E7
:106F0600253569256300256325352E326625630000
:106F16006D616E00737431007374320073743300E4
:106F2600737434007374350073743600706820000F
:106F3600636C200076722000686C2000617020006F
:106F4600727462006C616E0070702000706F690070
:106F560061632000006174200025632573002563AA
:106F660025332E30692563002534692563256300A2
:106F7600256325336925630025737C2563257325E1
:106F8600630020C0C0C0C0C0C7C0C0C0C0C0200011
:106F960025342E3066256300256325332E3066257D
:106FA6006300256325352E3066256300256325316C
:106FB600312E36667C25632531312E3666002563F3
:106FC6002532690025332E316625630020202020D6
:106FD6002020202020202020002020646973617258
:106FE6006D6564202000206E6F2074656C20636FD1
:106FF6006D2000206E6F2067707320666978200010
:1070060062617474207761726E696E670062617482
:1070160074637269746963616C00206261747420C0
:107026006572726F7220006C696E6B207175616C8F
:10703600697479006D6167207761726E696E6700A9
:107046006D616720637269746963616C00206D61AC
:107056006720206572726F7220002573002000B4CD
:10706600060000E803E803E803E8039DFF01640067
:107076000000007205FC327004730476047904B6CD
:107086002900070E091C1B1215383F363124232A06
:107096002D70777E796C6B6265484F464154535A22
:1070A6005DE0E7EEE9FCFBF2F5D8DFD6D1C4C3CA52
:1070B600CD90979E998C8B8285A8AFA6A1B4B3BAC2
:1070C600BDC7C0C9CEDBDCD5D2FFF8F1F6E3E4EDEF
:1070D600EAB7B0B9BEABACA5A28F88818693949D62
:1070E6009A2720292E3B3C35321F18111603040D12
:1070F6000A5750595E4B4C45426F68616673747D02
:107106007A898E878095929B9CB1B6BFB8ADAAA3AB
:10711600A4F9FEF7F0E5E2EBECC1C6CFC8DDDAD3A1
:10712600D4696E676075727B7C51565F584D4A43D1
:1071360044191E171005020B0C21262F283D3A3341
:10714600344E49404752555C5B7671787F6A6D6470
:10715600633E39303722252C2B0601080F1A1D14E1
:1071660013AEA9A0A7B2B5BCBB9691989F8A8D8491
:1071760083DED9D0D7C2C5CCCBE6E1E8EFFAFDF481
:10718600F3C2C0C0C1C0C0C1C0C0C4C0C0C1C0C0BD
:10719600C1C0C0C3C0C0C1C0C0C1C0C0C5C0C0C1DD
:1071A600C0C0C1C0C000000000CC2AFC323D2A6D20
:0E71B6002A9D2ABA2A532ADB29212B912B006D
:00000001FF
